:10000000EFC700000C9418080C9418080C941808FA
:100010000C9418080C9418080C9418080C941808E0
:100020000C9418080C9418080C9418080C941808D0
:10003000FFC700000C94DD3AFBC70000F9C70000C1
:10004000F7C700000C94FA4C0C949D20F1C70000F7
:100050000C945A22EDC70000EBC70000E9C700006E
:10006000E7C70000E5C70000E3C70000E1C70000E4
:10007000084AD73B3BCE016E84BCBFFDC12F3D6C0F
:1000800074319ABD56833DDA3D00C77F11BED9E475
:10009000BB4C3E916BAAAABE000000803F05A84C55
:1000A000CDB2D44EB93836A9020C50B99186880821
:1000B0003CA6AAAA2ABE000000803F4572726F7259
:1000C0003A005072696E7465722073746F70706557
:1000D000642064657520746F206572726F72732E70
:1000E0002046697820746865206572726F7220619D
:1000F0006E6420757365204D39393920746F207214
:10010000657374617274212E202854656D70657258
:1001100061747572652069732072657365742E2031
:10012000536574206974206265666F72652072651C
:100130007374617274696E6729005072696E7465B8
:10014000722068616C7465642E206B696C6C282960
:100150002063616C6C6564202121006F6B00526527
:1001600073656E643A006563686F3A002200556EED
:100170006B6E6F776E20636F6D6D616E643A2200F7
:100180007A5F6D696E3A00795F6D696E3A00785FEB
:100190006D696E3A005A3A00593A0020436F756E05
:1001A0007420583A00453A005A3A00593A00583AF1
:1001B000004649524D574152455F4E414D453A4DDB
:1001C00061726C696E2056313B20537072696E7497
:1001D00065722F6772626C206D617368757020663E
:1001E0006F722067656E36204649524D5741524521
:1001F0005F55524C3A687474703A2F2F7777772E88
:100200006D656E64656C2D70617274732E636F6DB5
:100210002050524F544F434F4C5F56455253494F15
:100220004E3A312E30204D414348494E455F545996
:1002300050453A4D656E64656C204558545255449E
:1002400045525F434F554E543A310A0020423A001E
:1002500020453A00543A0020573A0020453A0054CD
:100260003A0020403A0020423A006F6B20543A0096
:100270005072696E7465722073746F70706564205B
:1002800064657520746F206572726F72732E2046DC
:10029000697820746865206572726F7220616E647F
:1002A00020757365204D39393920746F207265735C
:1002B00074617274212E202854656D7065726174AA
:1002C0007572652069732072657365742E2053659D
:1002D00074206974206265666F726520726573743C
:1002E000617274696E6729006F6B004E6F204C69F4
:1002F0006E65204E756D6265722077697468206343
:100300006865636B73756D2C204C617374204C6948
:100310006E653A004E6F20436865636B73756D20A0
:1003200077697468206C696E65206E756D626572A0
:100330002C204C617374204C696E653A00636865CB
:10034000636B73756D206D69736D617463682C20C8
:100350004C617374204C696E653A004C696E65207F
:100360004E756D626572206973206E6F74204C61EA
:100370007374204C696E65204E756D6265722B3109
:100380002C204C617374204C696E653A002020501B
:100390006C616E6E657242756666657242797465EF
:1003A000733A20002046726565204D656D6F727945
:1003B0003A20006572696B00207C20417574686F7B
:1003C000723A2000323031322D30322D3235002059
:1003D0004C61737420557064617465643A20003117
:1003E0002E302E3020524332004D61726C696E3ACD
:1003F000200020536F6674776172652052657365C3
:100400007400205761746368646F67205265736578
:1004100074002042726F776E206F7574205265737E
:100420006574002045787465726E616C2052657346
:10043000657400506F7765725570007374617274E3
:10044000002200656E717565696E67202200656324
:10045000686F3A0020746F6F206C6F6E672065784C
:1004600074727573696F6E2070726576656E7465EF
:10047000640020636F6C6420657874727573696FB3
:100480006E2070726576656E7465640024F427D3FF
:10049000FD204D0FB0119A05160CE9022D09C80177
:1004A000650733013206DE005405A700AD04830062
:1004B0002A046900C10356006B03480023033D0072
:1004C000E6023500B1022D00840228005C02230000
:1004D0003902200019021C00FD011900E401170077
:1004E000CD011500B8011300A50111009401100001
:1004F00084010F0075010E0067010D005A010C0008
:100500004E010B0043010A0039010A002F010900C6
:10051000260109001D010800150107000E01080051
:1005200006010700FF000600F9000600F3000600C0
:10053000ED000600E7000500E2000500DD00050013
:10054000D8000500D3000400CF000500CA00040055
:10055000C6000400C2000400BE000300BB0004008B
:10056000B7000300B4000300B1000400AD000300B5
:10057000AA000300A7000200A5000300A2000300D8
:100580009F0002009D0003009A00020098000300F3
:100590009500020093000200910002008F0002000B
:1005A0008D0002008B00020089000200870002001B
:1005B000850002008300020081000100800002002B
:1005C0007E0002007C0001007B0002007900010037
:1005D000780002007600010075000100740002003E
:1005E0007200010071000100700002006E00010045
:1005F0006D0001006C0001006B0002006900010049
:10060000680001006700010066000100650001004C
:10061000640001006300010062000100610001004C
:10062000600001005F0001005E0001005D0001004C
:100630005C0001005B0000005B0001005A0001004B
:100640005900010058000100570000005700010048
:100650005600010055000100540000005400010044
:100660005300010052000100510000005100010040
:10067000500001004F0000004F0001004E0000003C
:100680004E0001004D0001004C0000004C00010034
:100690004B0000004B0001004A000100490000002F
:1006A0004900010048000000480001004700000028
:1006B0004700010046000000460001004500000020
:1006C0004500010044000000440001004300000018
:1006D0004300010042000000420001004100000010
:1006E0004100000041000100400000004000010006
:1006F0003F0000003F0001003E0000003E000000FF
:100700003E0001003D0000003D0001003C000000F3
:100710003C0000003C0001003B0000003B000000EA
:100720003B0001003A0000003A0000003A000100DE
:1007300039000000390000003900010038000000D5
:1007400038000000380001003700000037000000CA
:1007500037000100360000003600000036000100BE
:1007600035000000350000003500000035000100B4
:1007700034000000340000003400010033000000A9
:10078000330000003300000033000100320000009D
:100790003200000032000000320001003100000091
:1007A0003100000031000000310001003000000085
:1007B0003000000030000000300001002F00000079
:1007C0002F0000002F0000002F0001002E0000006D
:1007D0002E0000002E0000002E0000002E00010060
:1007E0002D0000002D0000002D0000002D00010054
:1007F0002C0000002C0000002C0000002C00000049
:100800002C0001002B0000002B0000002B0000003A
:100810002B0000002B0001002A0000002A0000002D
:100820002A0000002A0000002A0000002A0001001F
:100830002900000029000000290000002900000014
:100840002900000029000100280000002800000005
:1008500028000000280000002800010027000000F8
:1008600027000000270000002700000027000000EC
:1008700027000000270001002600000026000000DD
:1008800026000000260000002600000024F4B12805
:1008900073CB111D62AECC159698F410A287900D03
:1008A000127A190BF96E4009B965D307E65DB506F2
:1008B0003157D005615116054B4C7D04CE47FD03E1
:1008C000D14392033F403603093DE902203AA40296
:1008D0007C376A0212353602DC320802D430E1017C
:1008E000F32EBD01362D9E01982B8101172A670139
:1008F000B028500160273B0125262801FD24160160
:10090000E7230701E022F800E821EB00FD20DE00EC
:100910001F20D3004C1FC800841EBF00C51DB5009A
:10092000101DAD00631CA500BE1B9E00201B970080
:10093000891A9100F8198A006E198500E9187F005C
:100940006A187B00EF1776007917710008176D00A1
:100950009B166A0031166500CC1562006A155F00AF
:100960000B155B00B01458005814560002145200C6
:10097000B013500060134E0012134B00C712490011
:100980007E12460038124500F3114300B0114000BA
:1009900070113F0031113D00F4103C00B8103A00D6
:1009A0007E103800461037000F103500DA0F340083
:1009B000A60F3300730F3100420F3000120F3000CA
:1009C000E20E2D00B50E2D00880E2C005C0E2B00C3
:1009D000310E2A00070E2800DF0D2800B70D270072
:1009E000900D26006A0D2600440D2400200D2400E1
:1009F000FC0C2300D90C2200B70C2200950C21001E
:100A0000740C2000540C1F00350C1F00160C1F0026
:100A1000F70B1E00D90B1D00BC0B1C00A00B1C000B
:100A2000840B1C00680B1B004D0B1B00320B1A00C3
:100A3000180B1900FF0A1900E60A1900CD0A180060
:100A4000B50A18009D0A1800850A17006E0A1600DC
:100A5000580A1600420A16002C0A1600160A15003B
:100A6000010A1500EC091400D8091400C409140087
:100A7000B00914009C0913008909130076091300BA
:100A800063091200510912003F0912002D091100DB
:100A90001C0912000A091100F9081000E9081100E8
:100AA000D8081000C8081000B8081000A8081000E6
:100AB00098080F0089080F007A080F006B080F00D4
:100AC0005C080F004D080E003F080E0031080E00B4
:100AD00023080E0015080E0007080D00FA070D0088
:100AE000ED070D00E0070D00D3070D00C6070D0050
:100AF000B9070C00AD070C00A1070D0094070B000F
:100B000089070C007D070C0071070C0065070B00BE
:100B10005A070B004F070B0044070B0039070B0067
:100B20002E070B0023070B0018070A000E070B0007
:100B300003070A00F9060A00EF060A00E5060A00A4
:100B4000DB060A00D1060900C8060A00BE06090035
:100B5000B5060A00AB060900A206090099060900BD
:100B600090060900870609007E060900750609003F
:100B70006C060800640609005B06080053060900BD
:100B80004A060800420608003A0608003206080035
:100B90002A060800220608001A06080012060700A6
:100BA0000B06080003060800FB050700F405080013
:100BB000EC050700E5050700DE050700D70507007F
:100BC000D0050700C9050700C2050700BB050700DF
:100BD000B4050700AD050700A6050600A00507003F
:100BE00099050700920506008C050600860507009A
:100BF0007F05060079050600730507006C050600F1
:100C000066050600600506005A0506005405060044
:100C10004E05060048050600420505003D05060094
:100C200037050600310505002C05060026050500E0
:100C3000210506001B050500160506001005050028
:100C40000B0505000605060000050500FB04050070
:100C5000F6040500F1040500EC040500E7040500B6
:100C6000E2040500DD040500D8040500D3040500F6
:100C7000CE040500C9040500C4040500BF04040037
:100C8000BB040500B6040500B10405006563686F88
:100C90003A00205A3A0020593A0020583A00656E2E
:100CA0006473746F7073206869743A2000457272BF
:100CB0006F723A0054656D7065726174757265206B
:100CC0006865617465642062656420737769746324
:100CD000686564206F66662E204D415854454D501E
:100CE00020747269676765726564202121003A206B
:100CF000457874727564657220737769746368658A
:100D000064206F66662E204D494E54454D50207428
:100D100072696767657265642021003A20457874BE
:100D20007275646572207377697463686564206F97
:100D300066662E204D415854454D502074726967A7
:100D400067657265642021001000C90220013C0122
:100D500030020A014003EF005004DD006005D000BE
:100D60007006C5008007BC009008B500A009AE0061
:100D7000B00AA900C00BA300D00C9F00E00D9A00A0
:100D8000F00E96000010930010118F0020128C00BE
:100D900030138800401485005015820060168000D2
:100DA00070177D0080187A0090197800A01A7500DD
:100DB000B01B7300C01C7000D01D6E00E01E6C00E4
:100DC000F01F6A00002167001022650020236300E5
:100DD0003024610040255F0050265C0060275A00E7
:100DE0007028580080295600902A5400A02B5100EA
:100DF000B02C4F00C02D4D00D02E4B00E02F4800EE
:100E0000F0304600003243001033400020343D00F3
:100E100030353A0040363700503734006038300003
:100E200070392C00803A2800903B2200A03C1C0026
:100E3000B03D1400C03E0800D03F0000202D2049E6
:100E40006E76616C69642065787472756465722071
:100E50006E756D626572202100202D20496E7661CD
:100E60006C6964206578747275646572206E756D46
:100E7000626572210020403A006F6B20543A0050A6
:100E80004944204175746F74756E65206661696CA4
:100E9000656420212C2054656D70657261747572D3
:100EA0006520746F206869676800204B643A2000F1
:100EB000204B693A2000204B703A2000204E6F20D2
:100EC0006F76657273686F6F742000204B643A20F0
:100ED00000204B693A2000204B703A200020536FCD
:100EE0006D65206F76657273686F6F742000204B9C
:100EF000643A2000204B693A2000204B703A2000D1
:100F000020436C617369632050494420002054756C
:100F10003A2000204B753A2000206D61783A20007D
:100F2000206D696E3A200020643A200020626961D9
:100F3000733A2000002124272A002225282B002094
:100F4000232629020202020202020204040404040B
:100F50000404040303030303030303010101010168
:100F60000101010102040810204080010204081060
:100F7000204080010204081020408080402010089A
:100F80000402010000000102000000000000000453
:100F90000307060000000000000000000000000041
:100FA000000000494E46494E4954594E414ECDCC61
:100FB000CC3D0AD7233C17B7D13877CC2B32959547
:100FC000E6241FB14F0A000020410000C842004043
:100FD0001C4620BCBE4CCA1B0E5AAEC59D7477245D
:100FE00011241FBECFEFD0E1DEBFCDBF12E0A0E0E5
:100FF000B1E0E2E2F2EB02C005900D92A638B10733
:10100000D9F71AE0A6E8B2E001C01D92A73FB107E8
:10101000E1F71FE0C0EEDFE004C02297FE010E946E
:101020005D53CE3DD107C9F70E9498200C940F590B
:101030000C940000AF92BF92CF92DF92EF92FF929A
:101040000F931F93DF93CF93CDB7DEB7E0970FB623
:10105000F894DEBF0FBECDBFDE011196EFE6F2E0E1
:1010600080E101900D928150E1F7DE015196EFE5AC
:10107000F2E080E101900D928150E1F7DE0191965E
:10108000EFE4F2E080E101900D928150E1F7BE01C2
:101090006F5F7F4F40E255E021E1A22EB12CAC0EF4
:1010A000BD1E00E115E091E2E92EF12CEC0EFD1ED3
:1010B00080E3C82E85E0D82E20E030E0FB0181914E
:1010C0009191A191B191BF01FA0181939193A19363
:1010D000B193AF01F50181919191A191B1915F011E
:1010E000F80181939193A193B1938F01F7018191BD
:1010F0009191A191B1917F01F60181939193A19377
:10110000B1936F012F5F3F4F24303105B9F680E076
:1011100090E0AAEFB3E48093440590934505A09333
:101120004605B093470580E090E8ABE3B5E48093D3
:10113000480590934905A0934A05B0934B0580E07C
:1011400090E0DC018093400590934105A093420517
:10115000B093430520E23EE440E050E020930C05CC
:1011600030930D0540930E0550930F05809358055D
:1011700090935905A0935A05B0935B0580E090E0E9
:10118000A0EAB1E480934C0590934D05A0934E05E1
:10119000B0934F058DEC9CECACECBEE38093500516
:1011A00090935105A0935205B093530580E090E0D1
:1011B000A0EAB0E48093540590935505A09356059A
:1011C000B0935705E6E6F1E007C09091C00095FFA7
:1011D000FCCF8093C600319684918823B1F7E0E07C
:1011E000F1E006C09091C00095FFFCCF8093C6004F
:1011F00081918823B9F78091C00085FFFCCF8AE0F8
:101200008093C600E0960FB6F894DEBF0FBECDBF48
:10121000CF91DF911F910F91FF90EF90DF90CF90D2
:10122000BF90AF900895DF93CF9300D0CDB7DEB7D6
:101230008091F10A9091F20A9E012F5F3F4F009733
:1012400019F4275F3A4002C0281B390B3A832983DF
:1012500089819A810F900F90CF91DF910895AF927D
:10126000BF92CF92DF92EF92FF920F931F93CF9393
:10127000DF938BE095E040E052EC61E070E00E948B
:101280008F22EBE3F4E007C09091C00095FFFCCF04
:101290008093C600319684918823B1F78091C00075
:1012A00085FFFCCF8AE08093C60086E691E0FC01D2
:1012B00007C03091C00035FFFCCF2093C6003196A7
:1012C00024912223B1F724B720FF14C0E3E3F4E014
:1012D00007C04091C00045FFFCCF3093C600319657
:1012E00034913323B1F73091C00035FFFCCF3AE0A1
:1012F0003093C60021FF14C0E3E2F4E007C0409140
:10130000C00045FFFCCF3093C600319634913323A3
:10131000B1F73091C00035FFFCCF3AE03093C60002
:1013200022FF14C0E2E1F4E007C04091C00045FF95
:10133000FCCF3093C600319634913323B1F730910E
:10134000C00035FFFCCF3AE03093C60023FF14C045
:10135000E2E0F4E007C04091C00045FFFCCF3093CD
:10136000C600319634913323B1F73091C00035FF78
:10137000FCCF3AE03093C60025FF14C0E2EFF3E063
:1013800007C03091C00035FFFCCF2093C6003196D6
:1013900024912223B1F72091C00025FFFCCF2AE041
:1013A0002093C60014BEE9EEF3E007C03091C00000
:1013B00035FFFCCF2093C600319624912223B1F74C
:1013C000EFEDF3E007C03091C00035FFFCCF209374
:1013D000C600319624912223B1F72091C00025FF49
:1013E000FCCF2AE02093C600FC012491E6E6F1E060
:1013F00008C03091C00035FFFCCF2093C600319665
:1014000024912223B1F7EFECF3E007C03091C00044
:1014100035FFFCCF2093C600319624912223B1F7EB
:10142000E4ECF3E007C03091C00035FFFCCF20931F
:10143000C600319624912223B1F7E8EBF3E007C010
:101440003091C00035FFFCCF2093C6003196249127
:101450002223B1F7E3EBF3E007C03091C00035FF82
:10146000FCCF2093C600319624912223B1F720911E
:10147000C00025FFFCCF2AE02093C600FC01849128
:10148000E6E6F1E008C09091C00095FFFCCF8093A4
:10149000C600319684918823B1F7E4EAF3E007C0EF
:1014A0009091C00095FFFCCF8093C6003196849147
:1014B0008823B1F7B8DEBC018BE095E04AE050E04C
:1014C0000E949C23EDE8F3E007C09091C00095FFD7
:1014D000FCCF8093C600319684918823B1F78BE0CE
:1014E00095E060ED74E04AE050E00E949C2380911A
:1014F000C00085FFFCCF8AE08093C6001092740480
:1015000010927504109276041092770480E092DDB8
:10151000C0E3D5E000E215E03CE5E32E35E0F32E34
:101520006991799189919991F801A190B190C190B7
:10153000D1908F010E94DD4FA60195010E941252A9
:101540000E94B14FF70161937193819391937F0151
:10155000F5E0C034DF0721F70E94BA4B0E94CF2C80
:101560000E94D340DF91CF911F910F91FF90EF9098
:10157000DF90CF90BF90AF90089580916C049091D0
:101580006D04019660E070E00C94615380916C04EE
:1015900090916D04019660E070E04AE050E00C9498
:1015A000CE54682FE091EA02F091EB0240E650E061
:1015B000E49F9001E59F300DF49F300D1124C90187
:1015C00084519D4F70E00E9418569C0190936D04C9
:1015D00080936C0481E02115310509F480E00895C1
:1015E0000E94E2206093B4027093B5028093B60229
:1015F0009093B702EBE5F1E007C09091C00095FF32
:10160000FCCF8093C600319684918823B1F78091F6
:10161000C00085FFFCCF8AE08093C60008958BE070
:1016200095E00E94D222EEE5F1E007C09091C00063
:1016300095FFFCCF8093C600319684918823B1F743
:101640004091AC025091AD026091AE027091AF0238
:101650004F5F5F4F6F4F7F4F8BE095E02AE030E0A8
:101660000E946C238091C00085FFFCCF8AE08093AC
:10167000C600B6CF4F925F926F927F928F929F92E9
:10168000AF92BF92CF92DF92EF92FF920F931F9390
:10169000CF93DF9370E6C72ED12C64E0662E712CB9
:1016A00051E0A52EB12CE0E7F2E084904AE0942EC0
:1016B000E8EEF2E05490442443941CC28D3071F063
:1016C0008A3321F490916F04992341F020917004A2
:1016D000309171042F3531050CF4EEC1E0917004A6
:1016E000F0917104309719F410926F0422C2809126
:1016F0007204909173048C9DE0018D9DD00D9C9D92
:10170000D00D1124EC0FFD1FE451FD4F10822091EC
:101710006F04222309F0CBC110926F048C589B4FA9
:10172000FC0110828E0104511D4FC8016EE470E06F
:101730000E941856009709F412C190936D0480938B
:101740006C049501201B310B280F391F2C0F3D1FF6
:10175000C90184519D4F60E070E04AE050E00E9472
:10176000CE54609378047093790480937A049093B4
:101770007B04E090AC02F090AD020091AE021091BB
:10178000AF02A80197012F5F3F4F4F4F5F4F621786
:1017900073078407950709F43AC0209172043091C9
:1017A00073042C9DC0012D9D900D3C9D900D112426
:1017B00084519D4F68E171E00E942356009739F5EE
:1017C000EBEBF0E007C09091C00095FFFCCF809359
:1017D000C600319684918823B1F7EBE5F3E007C0AA
:1017E0009091C00095FFFCCF8093C6003196849104
:1017F0008823B1F78BE095E0B801A7012AE030E03B
:101800000E946C238091C00085FFFCCF92C0809124
:101810007204909173048C9DE0018D9DD00D9C9D70
:10182000D00D1124CE0184519D4F6AE270E00E94D8
:101830001856009709F457C020E000E002C00327C3
:101840002F5FFE01E20FF11DE451FD4F30813A326E
:10185000B1F790936D0480936C049E0124513D4F29
:10186000A501421B530B9A01280F391F2C0F3D1F56
:10187000C90184519D4F60E070E00E9461530E9455
:10188000AC4F10E00617170709F458C0EBEBF0E077
:1018900007C09091C00095FFFCCF8093C6003196A1
:1018A00084918823B1F7EDE3F3E007C09091C00085
:1018B00095FFFCCF8093C600319684918823B1F7C1
:1018C0004091AC025091AD026091AE027091AF02B6
:1018D0008BE095E02AE030E00E946C238091C0000C
:1018E00085FFFCCF26C0EBEBF0E007C09091C00075
:1018F00095FFFCCF8093C600319684918823B1F781
:10190000E4E1F3E007C09091C00095FFFCCF809325
:10191000C600319684918823B1F78BE095E0B80139
:10192000A7012AE030E00E946C238091C00085FF6F
:10193000FCCF8AE08093C60072DE47C080917804B5
:1019400090917904A0917A04B0917B048093AC02C9
:101950009093AD02A093AE02B093AF023BC0C8011A
:101960006AE270E00E9418560097A1F1EBEBF0E0FC
:1019700007C09091C00095FFFCCF8093C6003196C0
:1019800084918823B1F7EBEEF2E007C09091C0009C
:1019900095FFFCCF8093C600319684918823B1F7E0
:1019A0004091AC025091AD026091AE027091AF02D5
:1019B0008BE095E02AE030E00E946C238091C0002B
:1019C00085FFFCCF8AE08093C600109271041092CC
:1019D0007004AFC080917204909173048C9D80015B
:1019E0008D9D100D9C9D100D1124E801C451DD4FFB
:1019F000CE0167E470E00E941856009709F442C0D7
:101A000090936D0480936C0495012C1B3D0B280F63
:101A1000391F200F311FC90184519D4F60E070E0D4
:101A20000E9461530E94AC4F6430710558F580915B
:101A3000AB02882399F4852DE8EEF2E008C090917E
:101A4000C00095FFFCCF8093C60031968491882317
:101A5000B1F78091C00085FFFCCF12C0882DE0E770
:101A6000F2E008C09091C00095FFFCCF8093C600C3
:101A7000319684918823B1F78091C00085FFFCCF17
:101A80009092C60080917204909173040196B30104
:101A90000E94F752909373048093720480917C04A7
:101AA00090917D04019690937D0480937C04109224
:101AB0007104109270041EC08B3311F440926F04B5
:101AC00090916F049923B1F4409172045091730482
:101AD0004C9DF0014D9DF00D5C9DF00D1124E20F29
:101AE000F31FE451FD4F80832F5F3F4F309371040C
:101AF00020937004809107059091080520910905B5
:101B000030910A05821B930B8F779070009789F0B4
:101B100080917C0490917D048430910554F48BE095
:101B200095E00E94B62280936E048A3009F0C6CDFB
:101B3000D5CDDF91CF911F910F91FF90EF90DF9066
:101B4000CF90BF90AF909F908F907F906F905F905D
:101B50004F9008958F929F92AF92BF92CF92DF9253
:101B6000EF92FF920F931F93CF93DF93F1E1EF2E4C
:101B7000F2E0FF2ECDE8D2E008EC12E0E6E8CE2E4F
:101B8000E2E0DE2EF70181917F010BDD882321F158
:101B9000F4DC4B015C01F6018081882319F460912B
:101BA000D80201C061E070E0882777FD8095982F0A
:101BB0000E94DF4F288139814A815B810E94125245
:101BC0009B01AC01C501B4010E94644EF801608321
:101BD00071838283938309C088819981AA81BB81A3
:101BE000F80180839183A283B38324960C5F1F4FF7
:101BF0000894C11CD11CF5E1EF16F2E0FF0609F0D4
:101C0000C1CF86E4CEDC8823D1F0B7DC7B018C0128
:101C10006093D9027093DA028093DB029093DC0226
:101C200020E030E0A9010E944051181644F4E092EF
:101C3000F201F092F3010093F4011093F501DF91AA
:101C4000CF911F910F91FF90EF90DF90CF90BF90B9
:101C5000AF909F908F9008957DDF89E4A2DC882368
:101C600051F08BDC6093BC027093BD028093BE0286
:101C70009093BF020BC080E090E0DC018093BC0237
:101C80009093BD02A093BE02B093BF028AE489DCA8
:101C9000882351F072DC6093C0027093C10280937C
:101CA000C2029093C302089580E090E0DC0180932B
:101CB000C0029093C102A093C202B093C3020895E0
:101CC000CF92DF92EF92FF920F931F936091C80221
:101CD0007091C9028091CA029091CB0220E030E05D
:101CE000A9010E943D4F87FF0BC080E090E0DC011E
:101CF0008093C8029093C902A093CA02B093CB020A
:101D00006091CC027091CD028091CE029091CF0271
:101D100020E030E0A9010E943D4F87FF0BC080E02A
:101D200090E0DC018093CC029093CD02A093CE0290
:101D3000B093CF026091D0027091D1028091D20213
:101D40009091D30220E030E0A9010E943D4F87FF2F
:101D50000BC080E090E0DC018093D0029093D10230
:101D6000A093D202B093D3026091C8027091C902CD
:101D70008091CA029091CB0220E030E04DE453E420
:101D80000E944051181664F480E090E0ADE4B3E4A2
:101D90008093C8029093C902A093CA02B093CB0269
:101DA0006091CC027091CD028091CE029091CF02D1
:101DB00020E030E04DE453E40E944051181664F4F2
:101DC00080E090E0ADE4B3E48093CC029093CD0248
:101DD000A093CE02B093CF026091D0027091D10255
:101DE0008091D2029091D30220E030E040EF52E4A3
:101DF0000E944051181664F480E090E0A0EFB2E435
:101E00008093D0029093D102A093D202B093D302D8
:101E10000E94E2206093B4027093B5028093B602F0
:101E20009093B7026091EA017091EB01882777FDEA
:101E30008095982F0E94DF4F2091F2013091F3019D
:101E40004091F4015091F5010E94125220E030E0DF
:101E500040E752E40E94444F20E030E048EC52E476
:101E60000E94444F7B018C0188EC92E06CEC72E0A4
:101E700040ED52E024ED32E0A9EACA2EA2E0DA2ECB
:101E80000E945E2D8091C8029091C902A091CA0261
:101E9000B091CB0280938D0290938E02A0938F021B
:101EA000B09390028091CC029091CD02A091CE028D
:101EB000B091CF028093910290939202A0939302EB
:101EC000B09394028091D0029091D102A091D2025D
:101ED000B091D3028093950290939602A0939702BB
:101EE000B09398028091D4029091D502A091D6022D
:101EF000B091D7028093990290939A02A0939B028B
:101F0000B0939C021F910F91FF90EF90DF90CF90C4
:101F100008959F92AF92BF92CF92DF92EF92FF927D
:101F20000F931F93CF93DF93982E6091BC02709113
:101F3000BD028091BE029091BF022091C0023091FB
:101F4000C1024091C2025091C3020E944D517B01D7
:101F50008C016091EA017091EB0100D000D000D0BB
:101F6000CDB7DEB72196882777FD8095982F0E9400
:101F7000DF4F2091F2013091F3014091F401509133
:101F8000F5010E94125220E030E040E752E40E9446
:101F9000444F20E030E048EC52E40E94444F5B01A3
:101FA0006C01E882F9820A831B839C828091A902DA
:101FB0008D838DE892E068EC72E04CEB52E020E01B
:101FC00001E0B2E0EB2E0E9478248091C80290914B
:101FD000C902A091CA02B091CB0280938D02909366
:101FE0008E02A0938F02B09390028091CC029091C8
:101FF000CD02A091CE02B091CF0280939102909336
:102000009202A0939302B09394028091D002909197
:10201000D102A091D202B091D30280939502909305
:102020009602A0939702B09398028091D402909167
:10203000D502A091D602B091D702809399029093D5
:102040009A02A0939B02B0939C028DB79EB706960E
:102050000FB6F8949EBF0FBE8DBF0E94E220609322
:10206000B4027093B5028093B6029093B702DF91E9
:10207000CF911F910F91FF90EF90DF90CF90BF9085
:10208000AF909F900895F8940E94184C5A985A98CF
:102090005A985A98EBEBF0E007C09091C00095FF7A
:1020A000FCCF8093C600319684918823B1F7EAE390
:1020B000F1E007C09091C00095FFFCCF8093C6006F
:1020C000319684918823B1F78091C00085FFFCCFC1
:1020D0008AE08093C600FFCFEF92FF920F931F9389
:1020E0000E94E2202091B8023091B9024091BA02D8
:1020F0005091BB02E090B402F090B5020091B6029C
:102100001091B7026E197F09800B910B26173707C4
:102110004807590730F4211531054105510509F0EB
:10212000B2DF8091EE019091EF01A091F001B091AA
:10213000F1010097A105B10529F10E94E22020914B
:10214000B4023091B5024091B6025091B702621BC1
:10215000730B840B950B2091EE013091EF014091B0
:10216000F0015091F101261737074807590750F43D
:1021700090914C0A80914D0A981721F45A985A98D8
:102180005A985A980E94062D1EBA1F910F91FF90DF
:10219000EF9008952F923F924F925F926F927F92AD
:1021A0008F929F92AF92BF92CF92DF92EF92FF9267
:1021B0000F931F93DF93CF93CDB7DEB7A2970FB6E0
:1021C000F894DEBF0FBECDBF87E4EBD9882309F4B6
:1021D000A3C5D3D90E94AC4F6430710509F43CC04B
:1021E0006530710554F46230710531F16330710569
:1021F00054F577FF19C00C94F41F6A35710509F482
:1022000027C56B35710534F46C31710511F00C94F0
:10221000F41F64C06B35710509F41EC56C3571057A
:1022200011F00C94F41F1DC58091AB02882321F49A
:1022300091DC46DD0C9413208091AB02882319F4C5
:102240000BDD81E006C08091AB02882329F404DD18
:1022500080E05FDE0C94132080E5A3D9882341F051
:102260008CD90E94B14FE62EF72E082F192F03C0EC
:10227000EE24FF24870183E594D9882369F07DD972
:1022800020E030E04AE754E40E9412520E94B14F2D
:10229000E62EF72E082F192F0E9412410E94E220ED
:1022A0005B016C01AE0CBF1CC01ED11E0E94E2205F
:1022B0006093B4027093B5028093B6029093B70214
:1022C00004C00E94AB4381E007DF0E94E2206A1550
:1022D0007B058C059D05A8F30C94F41F8091F201F9
:1022E0009091F301A091F401B091F5018093DD028A
:1022F0009093DE02A093DF02B093E0028091EA01A6
:102300009091EB0190938B0280938A0284E690E097
:102310009093EB018093EA010E94E2206093B40263
:102320007093B5028093B6029093B70281E00E9449
:10233000D43A80918D0290918E02A0918F02B0913B
:1023400090028093C8029093C902A093CA02B093EE
:10235000CB028091910290919202A0919302B09150
:1023600094028093CC029093CD02A093CE02B093BE
:10237000CF028091950290919602A0919702B09120
:1023800098028093D0029093D102A093D202B0938E
:10239000D3028091990290919A02A0919B02B091F0
:1023A0009C028093D4029093D502A093D602B0935E
:1023B000D70280E090E0DC018093F2019093F3017A
:1023C000A093F401B093F50188E5EBD8882351F48C
:1023D00089E5E7D8882331F48AE5E3D8882311F426
:1023E00081E001C080E08093F60188E5DAD8882397
:1023F00009F4E6C089E5D5D8882309F4E1C080E076
:1024000090E0DC0180938D0290938E02A0938F0266
:10241000B09390028093910290939202A0939302C2
:10242000B09394028DE892E061E972E045E952E0F0
:1024300029E932E00E94453980E090ECA9E9B3EC4B
:102440008093C8029093C902A093CA02B093CB02B2
:102450008093CC029093CD02A093CE02B093CF0292
:102460002091DA013091DB014091DC015091DD01D6
:102470002093F2013093F3014093F4015093F5015E
:10248000E090DE01F090DF010091E0011091E101A8
:10249000C801B7010E943D4F87FF08C0E092F201DA
:1024A000F092F3010093F4011093F5016091F201B1
:1024B0007091F3018091F4019091F50120E030E0FA
:1024C00040E752E40E94444F7B018C0188EC92E08B
:1024D0006CEC72E040ED52E024ED32E0B9EACB2E34
:1024E000B2E0DB2E0E945E2D0E9412410F2EF0E022
:1024F0008F2EF0E09F2EF0E0AF2EF0E0BF2EF02DFB
:1025000080928D0290928E02A0928F02B0929002E1
:102510008092910290929202A0929302B0929402C1
:102520008DE892E061E972E045E952E029E932E0A4
:102530000E94453980918D0290918E02A0918F0268
:10254000B09190028093C8029093C902A093CA02EE
:10255000B093CB028091910290919202A09193024C
:10256000B09194028093CC029093CD02A093CE02BE
:10257000B093CF026091F2017091F3018091F40168
:102580009091F50120E030E040E752E40E94444F92
:102590007B018C0188EC92E06CEC72E040ED52E043
:1025A00024ED32E00E945E2D8092F2019092F301C0
:1025B000A092F401B092F5010E9412410E94CD3A1E
:1025C0008091F601882331F488E50E94D10A88239E
:1025D00009F4DEC00F2EF0E08F2EF0E09F2EF0E029
:1025E000AF2EF0E0BF2EF02D80928D0290928E02E1
:1025F000A0928F02B09290028DE892E061E972E0C1
:1026000045E952E029E932E00E94453980E090EC4A
:10261000A9E9B3EC8093C8029093C902A093CA02BF
:10262000B093CB026091DA017091DB018091DC0103
:102630009091DD016093F2017093F3018093F401B6
:102640009093F50120E030E040E752E40E94444FCF
:102650007B018C0188EC92E06CEC72E040ED52E082
:1026600024ED32E0A9EACA2EA2E0DA2E0E945E2D05
:102670000E94124180928D0290928E02A0928F024F
:10268000B09290028DE892E061E972E045E952E093
:1026900029E932E00E94453980E090E0A0EAB0E408
:1026A0008093C8029093C902A093CA02B093CB0250
:1026B0006091F2017091F3018091F4019091F50124
:1026C00020E030E040E752E40E94444F7B018C015F
:1026D00088EC92E06CEC72E040ED52E024ED32E0E8
:1026E0000E945E2D0E94124180E090E0A0E2B1ECD9
:1026F0008093C8029093C902A093CA02B093CB0200
:102700006091DA017091DB018091DC019091DD0133
:1027100020E030E040E05FE30E941252262F372F86
:10272000482F592F2093F2013093F3014093F40185
:102730005093F50120E030E040E752E40E94444F1E
:102740007B018C0188EC92E06CEC72E040ED52E091
:1027500024ED32E00E945E2D0E94124180928D0293
:1027600090928E02A0928F02B09290028092C80244
:102770009092C902A092CA02B092CB028092F2015A
:102780009092F301A092F401B092F5010E94CD3A2B
:102790008091F601882331F489E50E94D10A8823CB
:1027A00009F4DEC00F2EF0E08F2EF0E09F2EF0E057
:1027B000AF2EF0E0BF2EF02D809291029092920207
:1027C000A0929302B09294028DE892E061E972E0E7
:1027D00045E952E029E932E00E94453980E090EC79
:1027E000A9E9B3EC8093CC029093CD02A093CE02E2
:1027F000B093CF026091DE017091DF018091E00122
:102800009091E1016093F2017093F3018093F401E0
:102810009093F50120E030E040E752E40E94444FFD
:102820007B018C0188EC92E06CEC72E040ED52E0B0
:1028300024ED32E0F9EACF2EF2E0DF2E0E945E2D89
:102840000E9412418092910290929202A092930271
:10285000B09294028DE892E061E972E045E952E0BD
:1028600029E932E00E94453980E090E0A0EAB0E436
:102870008093CC029093CD02A093CE02B093CF026E
:102880006091F2017091F3018091F4019091F50152
:1028900020E030E040E752E40E94444F7B018C018D
:1028A00088EC92E06CEC72E040ED52E024ED32E016
:1028B0000E945E2D0E94124180E090E0A0E2B1EC07
:1028C0008093CC029093CD02A093CE02B093CF021E
:1028D0006091DE017091DF018091E0019091E10152
:1028E00020E030E040E05FE30E941252262F372FB5
:1028F000482F592F2093F2013093F3014093F401B4
:102900005093F50120E030E040E752E40E94444F4C
:102910007B018C0188EC92E06CEC72E040ED52E0BF
:1029200024ED32E00E945E2D0E94124180929102BD
:1029300090929202A0929302B09294028092CC0262
:102940009092CD02A092CE02B092CF028092F2017C
:102950009092F301A092F401B092F5010E94CD3A59
:102960008091F601882331F48AE50E94D10A8823F8
:1029700009F4DEC00F2EF0E08F2EF0E09F2EF0E085
:10298000AF2EF0E0BF2EF02D80929502909296022D
:10299000A0929702B09298028DE892E061E972E00D
:1029A00045E952E029E932E00E94453980E090E0B3
:1029B000A4E3B3EC8093D0029093D102A093D2020F
:1029C000B093D3026091E2017091E3018091E40140
:1029D0009091E5016093F2017093F3018093F4010B
:1029E0009093F50120E030E040E752E40E94444F2C
:1029F0007B018C0188EC92E06CEC72E040ED52E0DF
:102A000024ED32E0E9EACE2EE2E0DE2E0E945E2DD9
:102A10000E9412418092950290929602A092970293
:102A2000B09298028DE892E061E972E045E952E0E7
:102A300029E932E00E94453980E090E0A0E8BFE358
:102A40008093D0029093D102A093D202B093D3028C
:102A50006091F2017091F3018091F4019091F50180
:102A600020E030E040E752E40E94444F7B018C01BB
:102A700088EC92E06CEC72E040ED52E024ED32E044
:102A80000E945E2D0E94124180E090E0A0E0B0EC38
:102A90008093D0029093D102A093D202B093D3023C
:102AA0006091E2017091E3018091E4019091E50170
:102AB00020E030E040E05FE30E941252262F372FE3
:102AC000482F592F2093F2013093F3014093F401E2
:102AD0005093F50120E030E040E752E40E94444F7B
:102AE0007B018C0188EC92E06CEC72E040ED52E0EE
:102AF00024ED32E00E945E2D0E94124180929502E8
:102B000090929602A0929702B09298028092D00280
:102B10009092D102A092D202B092D3028092F2019E
:102B20009092F301A092F401B092F5010E94CD3A87
:102B300088E50E94D10A8823D9F00E94C60A61154F
:102B4000710581059105A1F00E94BD0A20919D02A9
:102B500030919E0240919F025091A0020E94644ECB
:102B600060938D0270938E0280938F0290939002F7
:102B700089E50E94D10A8823D9F00E94C60A61150E
:102B8000710581059105A1F00E94BD0A2091A10265
:102B90003091A2024091A3025091A4020E94644E7F
:102BA00060939102709392028093930290939402A7
:102BB0008AE50E94D10A8823D9F00E94C60A6115CD
:102BC000710581059105A1F00E94BD0A2091A50221
:102BD0003091A6024091A7025091A8020E94644E33
:102BE0006093950270939602809397029093980257
:102BF0008DE892E061E972E045E952E029E932E0CE
:102C00000E9445398091DD029091DE02A091DF02A1
:102C1000B091E0028093F2019093F301A093F4014C
:102C2000B093F50180918A0290918B029093EB0111
:102C30008093EA010E94E2206093B4027093B5028F
:102C40008093B6029093B7020E94CD3A0C94F41F81
:102C50001092D8020C94F41F81E08093D8020C9457
:102C6000F41F85E40E94D10A882311F40E941241C6
:102C700041E1842E42E0942E3DE9E32E32E0F32E32
:102C80000DE812E0AA24F40181914F010E94D10ABB
:102C90008823A9F10E94BD0AF70120813181428178
:102CA00053810E94644EF801608371838283938311
:102CB000FA2DF33061F40E94BD0AF801608371833C
:102CC0008283938389E992E00E94F23918C00E94BE
:102CD000BD0AF70120813181428153810E94644EF7
:102CE000F80160837183828393838DE892E061E9C8
:102CF00072E045E952E029E932E00E944539A394A7
:102D000024E030E0E20EF31E0C5F1F4F3A2D34300A
:102D100009F0B9CF0C94F41F8DE40E94D10A8823E6
:102D200011F40C944A1F0E94BD0A0E94AC4F6737F1
:102D3000710509F434C6683771050CF056C0653565
:102D4000710509F412C5663571051CF56A32710505
:102D500009F41BC16B32710574F46231710509F419
:102D6000C0C46F31710509F4A5C06131710511F05E
:102D70000C94F41F99C06335710509F4AEC4643531
:102D800071050CF0AEC46235710511F00C94F41F9E
:102D9000A1C46A36710509F473C46B36710574F405
:102DA0006836710509F434C1693671050CF0A1C1AA
:102DB0006C35710511F00C94F41FEDC46D3671057E
:102DC00009F429C26E36710534F46B36710511F0C1
:102DD0000C94F41F7CC46237710509F407C563378E
:102DE000710511F00C94F41FF3C46C3D710509F4E6
:102DF00028C76D3D71051CF56B3C710509F469C66A
:102E00006C3C710574F46E3B710509F49BC3693C1D
:102E1000710509F424C66C38710511F00C94F41F87
:102E200055C16D3C710509F491C66D3C71050CF4FA
:102E30006DC66E3C710511F00C94F41FE5C681E07F
:102E40006F32780709F4F9C791E06033790784F4A9
:102E5000E1E06D327E0709F415C7F1E06E327F07BD
:102E60000CF0E7C76D3D710511F00C94F41FFBC623
:102E700021E0653F720709F4F2C731E0663F73074E
:102E80003CF481E06039780711F00C94F41FE4C73A
:102E900091E0663F790709F4E4C7E3E0673E7E0707
:102EA00011F00C94F41FE1C75A9A5A9A5A9A5A9AF6
:102EB0000C94F41F0E94E2206093E1027093E202FE
:102EC0008093E3029093E4022091E5023091E602C0
:102ED0004091E7025091E802621B730B840B950B43
:102EE00028EE33E040E050E00E940A538DB79EB7D1
:102EF00008970FB6F8949EBF0FBE8DBF0DB71EB7D3
:102F00000F5F1F4FCE010196EDB7FEB7928381830D
:102F100083E291E0F80193838283CA01B9012CE333
:102F200030E040E050E00E940A53F80135832483EA
:102F3000778366830E943D56E6E6F1E084912DB7E3
:102F40003EB7285F3F4F0FB6F8943EBF0FBE2DBF70
:102F500008C09091C00095FFFCCF8093C6003196C9
:102F600084918823B1F7FE01319606C09091C0008C
:102F700095FFFCCF8093C60081918823B9F780919B
:102F8000C00085FFFCCF0C94F11F83E50E94D10A9D
:102F9000882311F40C94F41F0E94BD0A7B018C015C
:102FA00080E50E94D10A882311F40C94F41FC80113
:102FB000B7010E94AC4F8B0177FF02C00C94F41F45
:102FC0006F3F710519F014F00C94F41F0E94BD0AB4
:102FD0000E94AC4F7B01E5E1F2E0819191918E1569
:102FE0009F0511F40C94F41F32E0E938F307A9F7B8
:102FF000F7FE01C0F9C78E2D61E00E9403228E2DDD
:10300000602F0E9424228E2DB8010E947821ECC7E7
:103010008091A9028093E90284E50E94D10A882365
:1030200061F10E94BD0A0E94B14F6093E9026623DC
:1030300021F1E6E6F1E007C09091C00095FFFCCFDA
:103040008093C600319684918823B1F7E2E3F1E0E2
:1030500006C09091C00095FFFCCF8093C60081917F
:103060008823B9F78BE095E040E050E00E946623AA
:103070008091C00085FFFCCFB4C783E50E94D10AD0
:10308000882309F10E94BD0A7B018C01D090E902DE
:10309000AD2CBB240E94AC4FDC01CB016D2D0E94F6
:1030A000A041F501EE0FFF1FE755F54F9183808397
:1030B000F501EE0FFF1FEE0FFF1FEF54F54FE082FB
:1030C000F182028313830E94174C8EC783E50E940E
:1030D000D10A882309F488C70E94BD0A0E94AC4F18
:1030E000DC01CB010E9456429093AC0A8093AB0A5C
:1030F0007BC78091A9028093E90284E50E94D10AEE
:10310000882361F10E94BD0A0E94B14F6093E902D9
:10311000662321F1E6E6F1E007C09091C00095FF3B
:10312000FCCF8093C600319684918823B1F7E9E4FF
:10313000F1E006C09091C00095FFFCCF8093C600DF
:1031400081918823B9F78BE095E040E050E00E9440
:1031500066238091C00085FFFCCF43C7EAE6F2E01A
:1031600007C09091C00095FFFCCF8093C6003196B8
:1031700084918823B1F76091E902E62FF0E0EE0F29
:10318000FF1FE355F54F808191810E94A642AB015C
:10319000BC018BE095E022E030E00E947524E6E679
:1031A000F2E007C09091C00095FFFCCF8093C6006D
:1031B000319684918823B1F78091AF0A9091B00A3B
:1031C0000E94204BAB01BC018BE095E022E030E097
:1031D0000E947524E2E6F2E007C09091C00095FFDE
:1031E000FCCF8093C600319684918823B1F78091FB
:1031F000E90290E00E949A41BC018BE095E04AE030
:1032000050E00E949C238091C00085FFFCCF8AE0A3
:103210008093C60008C78091A9028093E90284E5E3
:103220000E94D10A882361F10E94BD0A0E94B14F19
:103230006093E902662321F1E6E6F1E007C0909190
:10324000C00095FFFCCF8093C600319684918823FF
:10325000B1F7E0E6F1E006C09091C00095FFFCCF29
:103260008093C60081918823B9F78BE095E040E018
:1032700050E00E9466238091C00085FFFCCFB1C65C
:1032800083E50E94D10A882309F10E94BD0A7B01CF
:103290008C01D090E902AD2CBB240E94AC4FDC0124
:1032A000CB016D2D0E94A041F501EE0FFF1FE755E8
:1032B000F54F91838083F501EE0FFF1FEE0FFF1F87
:1032C000EF54F54FE082F182028313830E94174C82
:1032D00079D75B016C018091E90290E0880F991F1A
:1032E000FC01E755F54F208031808355954FFC0157
:1032F0000190F081E02DF8A3EF8FEE24EA94FE2CEC
:103300008701EFE5F2E0249129A3EBE5F2E0449098
:10331000E7E5F2E034913AA35AE0552E04C189A1C1
:10332000EFE5F2E008C09091C00095FFFCCF8093DC
:10333000C600319684918823B1F76091E902E62FA7
:10334000F0E0EE0FFF1FE355F54F808191810E9461
:10335000A642AB01BC018BE095E022E030E00E9488
:103360007524842DEBE5F2E008C09091C00095FF34
:10337000FCCF8093C600319684918823B1F7609189
:10338000E9028BE095E070E04AE050E00E949C2367
:103390008AA1E7E5F2E008C09091C00095FFFCCF5C
:1033A0008093C600319684918823B1F717FF03C03C
:1033B000E7E7F1E026C006D79B01AC01C801B701E1
:1033C000605F784D8F4F9F4F621B730B840B950B83
:1033D00028EE33E040E050E00E940A538BE095E095
:1033E000BA01A9012AE030E00E9456238091C00072
:1033F00085FFFCCF0DC09091C00095FFFCCF80935E
:10340000C60081918823B9F78091C00085FFFCCF69
:103410005092C600D7D65B016C010E94AB4381E09D
:103420000E946C108FEFE8168FEFF8068FEF0807F9
:103430008FEF180751F58091E902EF8DF8A1E215A1
:10344000F30594F490E0880F991FFC01E755F54FC0
:103450008355954F20813181FC01808191818217B4
:1034600093070CF048C04CC090E0880F991FFC01F6
:10347000E755F54F8355954F20813181FC018081BF
:10348000918128173907BCF53BC017FD39C0609101
:10349000E902E62FF0E0EE0FFF1FE355F54F8081C4
:1034A00091810E94A6423B014C016091E902E62F06
:1034B000F0E0EE0FFF1FE755F54F808191810E94EC
:1034C000A6429B01AC01C401B3010E94634E0E945D
:1034D000AC4F262F372F482F592F57FF07C0509535
:1034E0004095309521953F4F4F4F5F4F2430310528
:1034F000410551052CF066D6E62EF72E082F192F20
:10350000FFEFEF16FFEFFF06FFEF0F07FFEF1F07BD
:1035100051F017FD6CC556D66E197F0927E2603150
:10352000720708F064C54ED66A197B098C099D099B
:10353000693E33E0730730E0830730E0930708F01B
:10354000EECE6BCF83E50E94D10A882361F00E9402
:10355000BD0A0E94AC4FDC01CB010E945642909301
:10356000AC0A8093AB0A2ED67B018C01E4E5F2E035
:10357000A490E0E5F2E08490ECE4F2E0D490EAE09C
:103580006E2E71C01FD66E197F09800B910B693E9C
:10359000E3E07E07E0E08E07E0E09E0708F45EC00F
:1035A0006091A902E62FF0E0EE0FFF1FE355F54F03
:1035B000808191810E94A642AB01BC018A2DE4E585
:1035C000F2E008C09091C00095FFFCCF8093C60048
:1035D000319684918823B1F78BE095E022E030E0CA
:1035E0000E947524882DE0E5F2E008C09091C000AB
:1035F00095FFFCCF8093C600319684918823B1F764
:103600006091A9028BE095E070E04AE050E00E94F2
:103610009C238D2DECE4F2E008C09091C00095FF52
:10362000FCCF8093C600319684918823B1F78091B6
:10363000AF0A9091B00A0E94204BAB01BC018BE015
:1036400095E022E030E00E9475248091C00085FF63
:10365000FCCF6092C600B6D57B018C010E94AB43C3
:1036600081E00E946C102091AB0A3091AC0A8091ED
:10367000AF0A9091B00A821793070CF483CFC0C4AD
:1036800083E50E94D10A8823F1F00E94BD0A20E060
:1036900030E0A9010E943D4F87FD0FC00E94BD0A86
:1036A00020E030E04FE753E40E94405118163CF010
:1036B0000E94BD0A0E94B14F03C060E001C06FEFDD
:1036C0006093AA0291C48FEF8093AA028DC41092D6
:1036D000AA028AC41092890287C481E08093890279
:1036E00083C483E50E94D10A882399F00E94BD0A11
:1036F00020E030E04AE754E40E9412520E94B14FA9
:103700006093EE017093EF018093F0019093F101CB
:103710006BC488E50E94D10A882309F07BC489E53F
:103720000E94D10A882309F075C48AE50E94D10A53
:10373000882309F06FC485E40E94D10A882309F028
:1037400069C40E9412415A980E947D414DC45A9802
:1037500089E50E94D10A81115A988AE50E94D10A0E
:10376000882309F441C45A983FC483E50E94D10AD2
:103770000E94BD0A20E030E04AE754E40E94125261
:103780000E94B14F6093B8027093B9028093BA025D
:103790009093BB0229C401E112E050E2E52E55E00E
:1037A000F52EF80181918F010E94D10A882339F00A
:1037B0000E94BD0AF701608371838283938324E0B2
:1037C00030E0E20EF31E32E00531130751F70CC46E
:1037D000E1EBF1E007C09091C00095FFFCCF809332
:1037E000C600319684918823B1F7FEC3EEEAF1E07A
:1037F00007C09091C00095FFFCCF8093C600319622
:1038000084918823B1F740918D0250918E0260918E
:103810008F02709190028BE095E022E030E00E94F0
:103820007524EBEAF1E007C09091C00095FFFCCF52
:103830008093C600319684918823B1F7409191021C
:103840005091920260919302709194028BE095E006
:1038500022E030E00E947524E8EAF1E007C0909190
:10386000C00095FFFCCF8093C600319684918823D9
:10387000B1F7409195025091960260919702709134
:1038800098028BE095E022E030E00E947524E5EAA2
:10389000F1E007C09091C00095FFFCCF8093C60077
:1038A000319684918823B1F74091990250919A0200
:1038B00060919B0270919C028BE095E022E030E0E9
:1038C0000E947524EBE9F1E007C09091C00095FFDC
:1038D000FCCF8093C600319684918823B1F70E9473
:1038E0006B410E94DF4F20912005309121054091CE
:1038F0002205509123050E94444FAB01BC018BE08F
:1039000095E022E030E0F1D7E8E9F1E007C09091DE
:10391000C00095FFFCCF8093C60031968491882328
:10392000B1F781E00E946B410E94DF4F2091240596
:103930003091250540912605509127050E94444F5E
:10394000AB01BC018BE095E022E030E0CED7E5E9A9
:10395000F1E007C09091C00095FFFCCF8093C600B6
:10396000319684918823B1F782E00E946B410E94D6
:10397000DF4F209128053091290540912A0550916B
:103980002B050E94444FAB01BC018BE095E022E087
:1039900030E0ABD78091C00085FFFCCF22C3EEE8BA
:1039A000F1E007C09091C00095FFFCCF8093C60066
:1039B000319684918823B1F783B180FD03C0EDE196
:1039C000F1E009C0E0E2F1E006C09091C00095FF8F
:1039D000FCCF8093C60081918823B9F7E7E8F1E036
:1039E00007C09091C00095FFFCCF8093C600319630
:1039F00084918823B1F7199903C0EDE1F1E009C082
:103A0000E0E2F1E006C09091C00095FFFCCF80930A
:103A1000C60081918823B9F7E0E8F1E007C09091F2
:103A2000C00095FFFCCF8093C60031968491882317
:103A3000B1F71A9903C0EDE1F1E009C0E0E2F1E06D
:103A400006C09091C00095FFFCCF8093C600819185
:103A50008823B9F78091C00085FFFCCFC2C241E145
:103A6000E42E42E0F42E00E010E0F70181917F01A6
:103A70000E94D10A882339F10E94BD0A30E3A32EA7
:103A800035E0B32EA00EB11E0E94B14FF501608348
:103A90007183828393830E94BD0A2CE5A22E25E0C8
:103AA000B22EA00EB11EF801E05EFA4F20813181E6
:103AB000428153810E9412520E94B14FF5016083EE
:103AC0007183828393830C5F1F4F0031110569F668
:103AD0008BC201E112E090E1E92E95E0F92EF801A8
:103AE00081918F010E94D10A882339F00E94BD0A7A
:103AF000F701608371838283938324E030E0E20ED8
:103B0000F31E32E00531130751F76EC283E50E94C0
:103B1000D10A882351F00E94BD0A60934405709336
:103B20004505809346059093470584E50E94D10A98
:103B3000882309F459C20E94BD0A60934805709316
:103B4000490580934A0590934B054EC283E50E9438
:103B5000D10A882351F00E94BD0A609340057093FA
:103B60004105809342059093430584E50E94D10A64
:103B7000882351F00E94BD0A60935805709359053F
:103B800080935A0590935B0582E40E94D10A8823B2
:103B900061F00E94BD0A0E94B14F60930C057093C2
:103BA0000D0580930E0590930F0588E50E94D10ABC
:103BB000882351F00E94BD0A60934C0570934D0517
:103BC00080934E0590934F058AE50E94D10A882381
:103BD00051F00E94BD0A6093500570935105809387
:103BE00052059093530585E40E94D10A882309F475
:103BF000FBC10E94BD0A60935405709355058093E4
:103C0000560590935705F0C101E112E08DE9E82EC9
:103C100082E0F82EF80181918F010E94D10A882359
:103C200039F00E94BD0AF701608371838283938318
:103C300024E030E0E20EF31E32E00431130751F7C6
:103C4000D3C183E50E94D10A882309F4CDC10E9423
:103C5000BD0A0E94AC4F7093EB016093EA0181E0D2
:103C600080938C02C1C183E50E94D10A882309F4A4
:103C7000BBC10E94BD0A0E94AC4F7093ED016093DE
:103C8000EC01B2C180E50E94D10A882351F00E9464
:103C9000BD0A6093FC017093FD018093FE01909337
:103CA000FF0189E40E94D10A882381F00E94BD0AA5
:103CB00025E93FEB46ED5DE30E941252609300025E
:103CC00070930102809302029093030284E40E94A5
:103CD000D10A882381F00E94BD0A25E93FEB46ED19
:103CE0005DE30E94444F6093040270930502809349
:103CF00006029093070283E40E94D10A882351F0C0
:103D00000E94BD0A609308027093090280930A0220
:103D100090930B020E948341E9E7F1E006C0909185
:103D2000C00095FFFCCF8093C60081918823B9F72E
:103D3000ECE7F1E006C09091C00095FFFCCF8093C6
:103D4000C60081918823B9F74091FC015091FD0193
:103D50006091FE017091FF018BE095E022E030E080
:103D6000C4D5E0E8F1E006C09091C00095FFFCCF1B
:103D70008093C60081918823B9F760910002709109
:103D80000102809102029091030225E93FEB46ED8A
:103D90005DE30E94444FAB01BC018BE095E022E063
:103DA00030E0A3D5E4E8F1E006C09091C00095FFB3
:103DB000FCCF8093C60081918823B9F760910402FB
:103DC00070910502809106029091070225E93FEB70
:103DD00046ED5DE30E941252AB01BC018BE095E021
:103DE00022E030E082D5E8E8F1E006C09091C00022
:103DF00095FFFCCF8093C60081918823B9F760912D
:103E000008027091090280910A0290910B0225E943
:103E10003FEB46ED5DE30E941252AB01BC018BE02B
:103E200095E022E030E061D58091C00085FFFCCFB5
:103E3000D8C081E00E940E3AD7C083E50E94D10A23
:103E4000882319F00E94BD0A04C060E070E086E19A
:103E500093E40E949845C8C00E941241C5C080E00A
:103E600001C081E00E941A08BFC01092AB0280918D
:103E7000B0029091B102A091B202B091B3028093CE
:103E8000AC029093AD02A093AE02B093AF020E9439
:103E90000F0BAAC084E50E94D10A882309F45DC0F3
:103EA0000E94BD0A0E94B14F6093E902E6E6F1E08C
:103EB000662369F107C09091C00095FFFCCF809305
:103EC000C600319684918823B1F7ECE8F1E006C092
:103ED0009091C00095FFFCCF8093C600819188230C
:103EE000B9F78BE095E040E050E0F0D3EEE8F1E088
:103EF00006C09091C00095FFFCCF8093C6008191D1
:103F00008823B9F78091C00085FFFCCF6AC010926A
:103F1000A90207C09091C00095FFFCCF8093C60016
:103F2000319684918823B1F7EFE9F1E006C09091D2
:103F3000C00095FFFCCF8093C60081918823B9F71C
:103F40006091A9028BE095E070E04AE050E0F4D384
:103F50008091C00085FFFCCF44C0E6E6F1E007C0D9
:103F60009091C00095FFFCCF8093C600319684915C
:103F70008823B1F7EEE6F1E007C09091C00095FF0D
:103F8000FCCF8093C600319684918823B1F72091AD
:103F9000EA023091EB0280E690E0289FF001299F31
:103FA000F00D389FF00D1124E451FD4F06C09091A3
:103FB000C00095FFFCCF8093C60081918823B9F79C
:103FC000ECE6F1E007C09091C00095FFFCCF809334
:103FD000C600319684918823B1F78091C00085FF97
:103FE000FCCF8AE08093C6000E94F00A1CC0EAD091
:103FF0006093E5027093E6028093E7029093E802F3
:10400000E1D06093B4027093B5028093B6029093AE
:10401000B702EACF0E94124188E50E94D10A8823A4
:1040200009F095CB95CBA2960FB6F894DEBF0FBEE4
:10403000CDBFCF91DF911F910F91FF90EF90DF9057
:10404000CF90BF90AF909F908F907F906F905F9038
:104050004F903F902F90089580917C0490917D0423
:104060008330910514F40E943A0B80917C04909166
:104070007D040097C1F00E94CA1080917C04909149
:104080007D04019790937D0480937C048091EA02E3
:104090009091EB02019664E070E00E94F7529093D9
:1040A000EB028093EA020E94AB4381E00E946C1015
:1040B0000C94113A0E94184C8091AB028823A1F510
:1040C00081E08093AB028091AC029091AD02A0910F
:1040D000AE02B091AF028093B0029093B102A09370
:1040E000B202B093B302EBEBF0E007C09091C000D6
:1040F00095FFFCCF8093C600319684918823B1F759
:10410000E2ECF0E007C09091C00095FFFCCF8093F7
:10411000C600319684918823B1F78091C00085FF55
:10412000FCCF8AE08093C60008958091AB02089589
:10413000A4D00E942F0990DFFECF1F920F920FB6DE
:104140000F9211242F933F938F939F93AF93BF931D
:104150008091820490918304A0918404B09185049D
:1041600030918604232F2A592D3720F02D570196A0
:10417000A11DB11D20938604809382049093830433
:10418000A0938404B093850480917E0490917F0471
:10419000A0918004B09181040196A11DB11D80936E
:1041A0007E0490937F04A0938004B0938104BF9118
:1041B000AF919F918F913F912F910F900FBE0F90D4
:1041C0001F9018958FB7F894209182043091830442
:1041D00040918404509185048FBFB901CA010895AC
:1041E0003FB7F89480917E0490917F04A091800461
:1041F000B091810426B5A89B05C02F3F19F0019608
:10420000A11DB11D3FBFBA2FA92F982F8827820F5C
:10421000911DA11DB11D9C01AD01220F331F441F33
:10422000551F280F391F4A1F5B1FB901CA01089586
:10423000EF92FF920F931F93CF93DF937B018C013B
:10424000CFDFEB010EC0CCDF6C1B7D0B83E0683E43
:10425000780738F00894E108F10801091109C851FC
:10426000DC4FE114F1040105110569F7DF91CF91ED
:104270001F910F91FF90EF900895789484B582601C
:1042800084BD84B5816084BD85B5826085BD85B5FA
:10429000816085BDEEE6F0E0808181608083E1E8A9
:1042A000F0E01082808182608083808181608083E1
:1042B000E0E8F0E0808181608083E1EBF0E08081E4
:1042C00084608083E0EBF0E0808181608083EAE7B6
:1042D000F0E080818460808380818260808380813F
:1042E000816080838081806880831092C1000895FE
:1042F0001F93CF93DF93182FEB0161E084D02097B9
:1043000009F44AC0CF3FD10509F449C0E12FF0E0DC
:10431000ED57F04FE491E330C1F0E43028F4E130A0
:1043200051F0E230B1F50CC0E63019F1E73049F157
:10433000E43079F514C084B5806884BDC7BD32C04F
:1043400084B5806284BDC8BD2DC080918000806826
:1043500080938000D0938900C093880023C080910F
:104360008000806280938000D0938B00C0938A008D
:1043700019C08091B00080688093B000C093B300F2
:1043800011C08091B00080628093B000C093B400EF
:1043900009C0C038D1051CF4812F60E002C0812F14
:1043A00061E052D0DF91CF911F910895833071F079
:1043B000843028F48130A1F0823021F514C0863099
:1043C000B1F08730D1F08430E9F404C080918000EE
:1043D0008F7703C0809180008F7D80938000089547
:1043E00084B58F7702C084B58F7D84BD0895809198
:1043F000B0008F778093B00008958091B0008F7DDA
:104400008093B000089590E0FC01ED59F04F2491A5
:10441000FC01ED5BF04FE491EE23A9F0F0E0EC5CE1
:10442000F04FA491B0E0662341F49FB7F8948C91CB
:10443000209582238C939FBF08959FB7F8948C9109
:10444000822B8C939FBF08950F931F93DF93CF937D
:104450000F92CDB7DEB7282F30E0F901ED57F04FBE
:104460008491F901ED59F04F14912D5B304FF90112
:1044700004910023C9F0882319F0698397DF6981CB
:10448000E02FF0E0E75CF04FA491B0E0662331F458
:104490009FB7F8948C911095812304C09FB7F8942E
:1044A0008C91812B8C939FBF0F90CF91DF911F91A7
:1044B0000F9108951F920F920FB60F9211242F9310
:1044C0003F934F935F936F938F939F93EF93FF93DC
:1044D0006091C6002091070530910805C901019639
:1044E0008F7790704091090550910A0584179507C0
:1044F00041F029573B4FF901608390930805809361
:104500000705FF91EF919F918F916F915F914F916F
:104510003F912F910F900FBE0F901F9018959A0109
:10452000AB0182E08093C00060E47BE48CE490E027
:104530000E942C532150304040405040CA01B901E4
:1045400022E030E040E050E00E942C533093C50060
:104550002093C400E1ECF0E0808180618083808161
:1045600088608083808180688083089580910905B8
:1045700090910A0520910705309108052817390701
:1045800069F0FC01E957FB4F208101968F7790700D
:1045900090930A058093090530E002C02FEF3FEFAA
:1045A000C90108958091090590910A059093080525
:1045B0008093070508956F927F928F929F92AF929A
:1045C000BF92CF92DF92EF92FF920F931F93DF93F0
:1045D000CF93CDB7DEB7A0970FB6F894DEBF0FBE6E
:1045E000CDBF5C01CB01BA01611571058105910553
:1045F00031F4C50160E340E050E0A6D042C06E0156
:104600000894C11CD11CEE24FF248701622E77245C
:1046100088249924A40193010E940A53F60161930E
:104620006F010894E11CF11C011D111DB901CA01A3
:10463000611571058105910569F7D801C7010197D9
:10464000A109B1096E010894C11CD11CC80ED91E64
:1046500013C0F60160816A3010F4605D01C0695CCE
:10466000C50140E050E070D00894E108F10801096C
:1046700011090894C108D108E114F10401051105DC
:1046800041F7A0960FB6F894DEBF0FBECDBFCF9115
:10469000DF911F910F91FF90EF90DF90CF90BF902F
:1046A000AF909F908F907F906F9008952115310566
:1046B00039F48091C00085FFFCCF4093C600089577
:1046C0007ACF9A01AB0160E070E0F0CF9A01462FFB
:1046D00050E060E070E0EACFEF92FF920F931F93FB
:1046E000CF93DF93EC017A018B012115310539F469
:1046F0008091C00085FFFCCFE092C60016C02A3032
:10470000310591F477FF0CC06DE240E050E01CD021
:1047100010950095F094E094E11CF11C011D111D11
:10472000CE01B801A7012AE046DFDF91CF911F91AA
:104730000F91FF90EF9008959A01FB01AF0166275A
:1047400057FD6095762FC8CF9A01462F50E060E064
:1047500070E0C2CFCF93DF93EC016DE040E050E01A
:10476000F3DFCE016AE040E050E0EEDFDF91CF9171
:104770000895CF93DF93EC01A4DFCE01EBDFDF914F
:10478000CF9108958F929F92BF92CF92DF92EF9236
:10479000FF920F931F93CF93DF934C017A018B010C
:1047A000D22ECB01BA0120E030E0A9010E943D4F9A
:1047B00087FF09C0C4016DE240E050E0C5DF17FB90
:1047C000109517F91095C0E050E040E030E02FE37D
:1047D00011C0DA01F9016B2F742F8F2F922F20E077
:1047E00030E040E251E40E94444F562F472F382FCB
:1047F000292FCF5FCD1568F3C801B701DA01F901A0
:104800002B2F342F4F2F5E2F0E94644EC62EF72E73
:104810008C01912F0E94B14FC62FE72ED82FB92EB1
:104820000E94DD4F9B01AC016C2D7F2D802F912FBD
:104830000E94634EC62EF72E182F092FC4014C2F4D
:104840005E2D6D2F7B2D2AE030E030DFDD2009F476
:104850003EC0E1EBF1E006C09091C00095FFFCCFB7
:104860008093C60081918823B9F731C098016C2DDF
:104870007F2D832F902F20E030E040E251E40E9412
:1048800012528B01F82EE92E9701712F832F922F50
:104890000E94AC4F9B01AC01EB01C401B9014AE09D
:1048A00050E04ADFBE01882777FD8095982F0E944F
:1048B000DF4F9B01AC01F701602F712F8F2F9E2FCF
:1048C0000E94634EC62EF72E182F092FDA94DD2092
:1048D00069F6DF91CF911F910F91FF90EF90DF90DC
:1048E000CF90BF909F908F9008954CCF08950895DA
:1048F0002F923F924F925F926F927F928F929F92F0
:10490000AF92BF92CF92DF92EF92FF920F931F93DD
:10491000DF93CF93CDB7DEB7C055D0400FB6F89434
:10492000DEBF0FBECDBF4C017A8F698F3A012AA737
:104930000EABEFAAA8AEB9AECAAEDBAE022F10E046
:10494000000F111F000F111F9301200F311F3BABF0
:104950002AABD9012D903D904D905C90FC01E00F69
:10496000F11FC201B10120813181428153810E9436
:10497000644E6CAF7DAF8EAF9FAFBEA9EB2EFF2410
:10498000EE0CFF1CEE0CFF1CF301EE0DFF1DFDAB4A
:10499000ECABA080B180C280D380F401EE0DFF1D8E
:1049A000C601B50120813181428153810E94644E4C
:1049B00021966FAF219722967FAF229723968FAFD4
:1049C000239724969FAF2497FFA98F2F90E0880FFD
:1049D000991F880F991FF401E80FF91F2081318179
:1049E000428153812B8F3C8F4D8F5E8F498D5A8D25
:1049F000840F951FDC016D917D918D919C912B8D84
:104A00003C8D4D8D5E8D0E94634E262F372F482F93
:104A1000592F2F8F38A349A35AA3E98DFA8D3C96BD
:104A20002996FFAFEEAF2997A98DBA8D1C962D91CF
:104A30003D914D915C911F972EA73FA748AB59AB75
:104A4000D4011C962D913D914D915C911F972BA304
:104A50003CA34DA35EA3A20191015058298B3A8B30
:104A60004B8B5C8B1501260157FA509457F85094E4
:104A7000E98DFA8DE00FF11F608171818281938150
:104A8000BCADADADFEADEFAD2B2F3A2F4F2F5E2F4E
:104A90000E94634EB62EA72E882E692EE98DFA8DC0
:104AA000EE0DFF1D60817181828193812196BFADE2
:104AB00021972296AFAD22972396FFAD2397249698
:104AC000EFAD24972B2F3A2F4F2F5E2F0E94634E6E
:104AD0008B01F82EE92E69897A898B899C89F701E7
:104AE000202F312F4F2F5E2F0E9412526D8B7E8B05
:104AF0008F8B988FC201B101D5012B2F3A2F482DF2
:104B0000562D0E9412529B01AC016D897E898F89BE
:104B1000988D0E94634E6D8B7E8B8F8B988F6989E9
:104B20007A898B899C89D5012B2F3A2F482D562DB8
:104B30000E9412525B016C01C201B101F701202FEA
:104B4000312F4F2F5E2F0E9412529B01AC01C601E4
:104B5000B5010E94644E9B01AC016D897E898F89ED
:104B6000988D0E94D74E162F072FF82EE92EA801F8
:104B70009701652F742F832F922F20E030E0A90139
:104B80000E943D4F87FF10C0A8019701652F742F29
:104B9000832F922F2BED3FE049EC50E40E94644EAE
:104BA000162F072FF82EE92EAA968FADAA978823E5
:104BB00081F0A8019701652F702F832F9E2D2BED7B
:104BC0003FE049EC50E40E94634E162F072FF82E69
:104BD000E92EA8019701652F702F832F9E2DA9968E
:104BE0002CAD3DAD4EAD5FADA9970E9412522F8DF9
:104BF00038A149A15AA15F770E944D515B016C0118
:104C00002FE632E143E85AE30E943D4F87FDA6C2FA
:104C1000C601B5010E941A500E94B14F7DA76CA732
:104C20006115710521F481E090E09DA78CA7ACA5EA
:104C3000BDA5BD0180E090E00E94DD4F5B016C01ED
:104C4000A8019701652F702F832F9E2DA601950136
:104C50000E94444F6D8B7FA388A799A76F8D78A181
:104C600089A19AA1A60195010E94444F2A966FAF8F
:104C70002A972B967FAF2B972C968FAF2C972D963C
:104C80009FAF2D976EA57FA588A999A92BA13CA1BF
:104C90004DA15EA10E94634EA60195010E94444F62
:104CA0002E966FAF2E972F967FAF2F9760968FAF70
:104CB000609761969FAF61975D894FA138A529A53F
:104CC000652F742F832F922F20E030E040E05FE3C8
:104CD0000E941252BD89AFA1F8A5E9A52B2F3A2F4A
:104CE0004F2F5E2F0E9412529B01AC0160E070E0DA
:104CF00080E89FE30E94634E6EA725967FAF2597BD
:104D000026968FAF269727969FAF2797BFA9EB2FA1
:104D1000F0E0EE0FFF1FEE0FFF1FCE010196E80F30
:104D2000F91F2B8D3C8D4D8D5E8D20833183428309
:104D300053832BA13CA14DA15EA12D873E874F87B8
:104D4000588BBB2441E050E05CA34BA3BAA5AB2F2A
:104D5000B0E0AA0FBB1FAA0FBB1F9C012A0F3B1F6D
:104D60003C8F2B8F5EA9452F50E0440F551F440FF9
:104D7000551F81E090E08C0F9D1F840F951F98A315
:104D80008F8FFBA7EAA7CAC19B2D99310CF068C091
:104D900069897A898B899C89BD89AFA1F8A5E9A524
:104DA0002B2F3A2F4F2F5E2F0E9412527B018C0126
:104DB000C201B101BEA52596AFAD25972696FFADE0
:104DC00026972796EFAD27972B2F3A2F4F2F5E2F41
:104DD0000E9412529B01AC01C801B7010E94644EAF
:104DE000D62EA72E882E692E69897A898B899C896F
:104DF000BEA52596AFAD25972696FFAD269727969B
:104E0000EFAD27972B2F3A2F4F2F5E2F0E94125274
:104E1000162F072FF82EE92EC201B101BD89AFA1CF
:104E2000F8A5E9A52B2F3A2F4F2F5E2F0E94125283
:104E30009B01AC01D801F7016B2F7A2F8F2F9E2F8A
:104E40000E94634E262F372F482F592F298B3A8BDC
:104E50004B8B5C8BB3942D2C3A2C482C562C6AC06F
:104E6000ABA1BCA1BD0180E090E00E94DD4FBD89F7
:104E7000AFA1F8A5E9A52B2F3A2F4F2F5E2F0E9447
:104E800012527B018C017F2D912F0E94414F1B01FB
:104E90002C016E2D7F2D802F912F0E9475525B016A
:104EA0006C01EAA9FBA9E080F1800281138117FB64
:104EB000109517F91095ACA9BDA96D907D908D90B6
:104EC0009C90C801B701A20191010E941252698B06
:104ED0007A8B8B8B9C8BC401B301A60195010E9438
:104EE00012529B01AC0169897A898B899C890E9445
:104EF000644E262F372F482F592F298B3A8B4B8BF7
:104F00005C8BC801B701A60195010E9412527B017A
:104F10008C01C401B301A20191010E9412529B01B4
:104F2000AC01C801B7010E94634E262E372E482ED1
:104F3000592EBB245CAD4DAD3EAD2FAD652F742F0A
:104F4000832F922F29893A894B895C890E94644E6C
:104F5000EB8DFC8D608371838283938321965FAD9B
:104F6000219722964FAD229723963FAD2397249603
:104F70002FAD2497652F742F832F922FA2019101BB
:104F80000E94644EAF8DB8A16D937D938D939C93D9
:104F90001397EAA5FBA560817181828193812A968E
:104FA000BFAD2A972B96AFAD2B972C96FFAD2C97C4
:104FB0002D96EFAD2D972B2F3A2F4F2F5E2F0E945E
:104FC000644EAAA5BBA56D937D938D939C93139777
:104FD0006D857E858F8598892E96BFAD2E972F96ED
:104FE000AFAD2F976096FFAD60976196EFAD61977B
:104FF0002B2F3A2F4F2F5E2F0E94644E6D877E8796
:105000008F87988B69817A818B819C8120E030E049
:10501000A9010E943D4F87FF07C080E090E0DC01BE
:1050200089839A83AB83BC836D817E818F819885D0
:1050300020E030E0A9010E943D4F87FF07C080E0DB
:1050400090E0DC018D839E83AF83B88769857A8584
:105050008B859C8520E030E0A9010E943D4F87FFB1
:1050600007C080E090E0DC0189879A87AB87BC8726
:1050700069817A818B819C8120E030E04DE453E4AA
:105080000E944051181644F480E090E0ADE4B3E48F
:1050900089839A83AB83BC836D817E818F81988560
:1050A00020E030E04DE453E40E944051181644F4EF
:1050B00080E090E0ADE4B3E48D839E83AF83B88756
:1050C00069857A858B859C8520E030E040EF52E44D
:1050D0000E944051181644F480E090E0A0EFB2E442
:1050E00089879A87AB87BC87CE010196BE016B5F2B
:1050F0007F4FAE01475F5F4F9E01235F3F4FE8AC9C
:10510000F9AC0AAD1BADFAE6CF2ED12CCC0EDD1ECC
:10511000D5D4EBA1FCA13196FCA3EBA32BA13CA120
:105120004CA55DA52417350708F42ECE698D7A8D20
:105130006C5F7F4F498D5A8D485F5F4F898D9A8D87
:1051400029962EAD3FAD2997E8ACF9AC0AAD1BAD61
:10515000EAE6CE2ED12CCC0EDD1EB0D4C05BDF4FE4
:105160000FB6F894DEBF0FBECDBFCF91DF911F9178
:105170000F91FF90EF90DF90CF90BF90AF909F90F6
:105180008F907F906F905F904F903F902F900895F9
:105190008F5F803109F480E008952F923F924F9203
:1051A0005F926F927F928F929F92AF92BF92CF92B7
:1051B000DF92EF92FF920F931F93DF93CF93CDB7C0
:1051C000DEB76A970FB6F894DEBF0FBECDBF9A8FD9
:1051D000898F3A014B0178018901DC01D8966D91E4
:1051E0007D918D919C91DB970E94DD4F5B016C015D
:1051F000A40193010E9412520E942A4F0E94B14FB3
:10520000262F372F482F592F2D873E874F87588BB2
:10521000C601B501A80197010E9412520E942A4FAF
:105220000E94B14F9B01AC01298B3A8B4B8B5C8B5D
:105230008D859E85AF85B88988379105A105B10513
:1052400040F488E790E0A0E0B0E08D879E87AF87CC
:10525000B88B283731054105510540F428E730E087
:1052600040E050E0298B3A8B4B8B5C8BE98DFA8DBB
:10527000EC5BFF4F6080718082809380A98DBA8D36
:10528000DC966D917D918D919C91DF970E94DD4F11
:105290006D837E838F839887C401B3010E94DF4FA3
:1052A0001B012C0120E030E0A9010E943D4F882322
:1052B00029F1C601B501A60195010E9412527B0198
:1052C0008C016D817E818F8198859B01AC010E944C
:1052D00012529B01AC01C801B7010E94634E7B01D1
:1052E0008C01C201B101A20191010E94644E9B0197
:1052F000AC01C801B7010E94444F04C060E070E0F7
:1053000080E090E00E942A4F0E94AC4F69837A832C
:105310008B839C83E980FA800B811C81E98DFA8D57
:10532000E05CFF4F60817181828193810E94DD4F3B
:1053300069877A878B879C8766277727CB016619D1
:105340007709880999090E94DF4F3B014C0120E051
:1053500030E0A9010E943D4F882349F169857A8593
:105360008B859C859B01AC010E9412526D8B7E8BBC
:105370008F8B988FC601B501A60195010E9412522C
:105380009B01AC016D897E898F89988D0E94634E47
:105390005B016C01C401B301A40193010E94644E3E
:1053A0009B01AC01C601B5010E94444F04C060E0FE
:1053B00070E080E090E00E941A50E98DFA8DA0889C
:1053C000B188C288D3883501460129813A814B8151
:1053D0005C81621A730A840A950A0E94AC4FA40188
:1053E0009301261B370B480B590BDA01C90157FFF4
:1053F00068C0C201B10120E030E0A9010E943D4F28
:10540000882309F443C0C201B101A20191010E94A5
:10541000644E7B018C01C601B5010E94DD4F9B01EA
:10542000AC01C801B7010E9412527B018C016D8151
:105430007E818F8198859B01AC010E9412529B0155
:10544000AC01C801B7010E94634E7B018C016985E4
:105450007A858B859C859B01AC010E9412529B0131
:10546000AC01C801B7010E94644E7B018C01C201EE
:10547000B10120E030E040E850E40E9412529B016C
:10548000AC01C801B7010E94444F04C060E070E065
:1054900080E090E00E942A4F0E94AC4FE62EF72E4B
:1054A000082F192F17FF03C0EE24FF248701EA14E9
:1054B000FB040C051D0510F08601750180E090E0ED
:1054C000DC012FB7F894E98DFA8DE45BFF4F308152
:1054D000332311F5E98DFA8DE48AF58A068B178B53
:1054E000E80EF91E0A1F1B1FE08EF18E028F138F2C
:1054F0008D859E85AF85B88984AF95AFA6AFB7AFD0
:10550000AF01405C5F4F89899A89AB89BC89FA01F8
:1055100080839183A283B3832FBF6A960FB6F894DA
:10552000DEBF0FBECDBFCF91DF911F910F91FF90D6
:10553000EF90DF90CF90BF90AF909F908F907F9033
:105540006F905F904F903F902F900895AF92BF92D1
:10555000CF92DF92EF92FF920F931F93CF93DF933F
:10556000EB018A01209709F472C04115510509F435
:105570006EC0DAA4CBA4BCA4ADA46EA17FA188A503
:1055800099A5D601F5012B2F3A2F4F2F5E2F0E94A0
:105590003D4F882309F45BC08FA9882309F04BC0D5
:1055A000F801E6A0F7A000A511A5A6019501652FB9
:1055B000742F832F922FA80197010E944051181633
:1055C000D4F5C801B701A80197010E9412527B01CE
:1055D0008C012AA93BA94CA95DA95058CA01B9015F
:1055E0000E94644E2EA53FA548A959A90E941252B7
:1055F0009B01AC01C801B7010E94634E0E947F521B
:10560000E62E172F082FF92EA6019501652F742F6E
:10561000832F922F2E2D312F402F5F2D0E943D4F33
:1056200087FF04C0ED2C1C2D0B2DFA2C5E2D412F75
:10563000302F2F2D02C0A6019501852F942FA32F67
:10564000B22F8EA39FA3A8A7B9A781E08EABDF914D
:10565000CF911F910F91FF90EF90DF90CF90BF906F
:10566000AF900895CF92DF92EF92FF920F931F9326
:10567000DF93CF930F92CDB7DEB780914C0A809124
:105680004C0A20914D0A90E04096821B91098F7040
:1056900090708430910544F120914C0A23502F7072
:1056A00040E050E000E010E08DE4E82EF12C18C05E
:1056B000222309F420E12150822F90E08E9D600189
:1056C0008F9DD00C9E9DD00C11248CE795E0C80EC8
:1056D000D91EC601B801298339DFA80186012981B5
:1056E00080914D0A281721F70F90CF91DF911F91DC
:1056F0000F91FF90EF90DF90CF9008958F929F923F
:10570000AF92BF92CF92DF92EF92FF920F931F93CF
:10571000CF93DF93EC016B01009709F467C08FA969
:10572000882309F063C0EEA0FFA008A519A5FB011E
:10573000B6A0A7A090A481A4C801B701D501F40127
:105740002B2F3A2F4F2F5E2F0E943D4F87FF4EC0C9
:10575000C801B701A80197010E9412527B018C0178
:105760002AA93BA94CA95DA95058CA01B9010E94B8
:10577000644E2EA53FA548A959A90E9412529B012B
:10578000AC01C801B7010E94634E0E947F52E62E11
:10579000C72FD82F192FA5019401652F742F832FA0
:1057A000922F2E2D3C2F4D2F512F0E943D4F87FFC2
:1057B00004C0EB2CCA2DD92D182DA5019401652FFD
:1057C0007A2D832F982D2E2D3C2F4D2F512F0E9457
:1057D0003D4F882359F08E2D9C2FAD2FB12FF60110
:1057E00086A397A3A0A7B1A781E086ABDF91CF9155
:1057F0001F910F91FF90EF90DF90CF90BF90AF90EF
:105800009F908F900895DF92EF92FF920F931F93D6
:10581000CF93DF93D0904D0A00E010E080E090E05D
:105820002DE4E22EF12C13C02D2D30E02E9DE00151
:105830002F9DD00D3E9DD00D1124C458DA4FB801D4
:10584000AE015CDF8D2DA4DCD82EC8018E01209125
:105850004C0AD21649F7B80140E050E04FDFDF9123
:10586000CF911F910F91FF90EF90DF9008952F92AD
:105870003F924F925F926F927F928F929F92AF92E0
:10588000BF92CF92DF92EF92FF920F931F93CF932D
:10589000DF93F0904D0AC0E0D0E03DE4632E712C20
:1058A0003EC0069D6001079DD00C169DD00C1124B2
:1058B0008CE795E0C80ED91E209769F18EA9882340
:1058C00021F4F60186A9882331F18AA09BA0ACA01F
:1058D000BDA06EA17FA188A599A5A50194010E94F4
:1058E000444F1B012C01069DF001079DF00D169DF4
:1058F000F00D1124E458FA4F66A177A180A591A577
:10590000A50194010E94444F8B019C01CE01B2017C
:10591000A10143DC1EAA8F2D3BDCF82EE6010F2DE2
:10592000112707FD109580914C0A90E00817190780
:1059300009F0B7CF2097E9F0CAA0DBA0ECA0FDA04A
:105940006EA17FA188A599A5A70196010E94444F49
:105950004B015C016DEC7CEC8CE49DE3A7019601AE
:105960000E94444F8B019C01CE01B501A40115DCBE
:105970001EAADF91CF911F910F91FF90EF90DF90C2
:10598000CF90BF90AF909F908F907F906F905F90DF
:105990004F903F902F90089565DE35DF68CF1092CD
:1059A0004C0A10924D0A80E1ECE6F5E0DF011D9211
:1059B0008A95E9F780E090E0DC018093530A9093A8
:1059C000540AA093550AB093560A8093570A9093AD
:1059D000580AA093590AB0935A0A80935B0A90938D
:1059E0005C0AA0935D0AB0935E0A80935F0A90936D
:1059F000600AA093610AB093620A80934F0A909361
:105A0000500AA093510AB093520A0895CF939091EF
:105A10004D0A80914C0A981779F140914D0A242F34
:105A200030E08DE490E0289FF001299FF00D389F31
:105A3000F00D1124EC53FA4FC08150E02DE430E01A
:105A400016C0842F90E0829FF001839FF00D929FFB
:105A5000F00D1124EC53FA4F80819181A281B38122
:105A60000097A105B10509F05F5F4F5F4F7080910E
:105A70004C0A481731F70AC06091AA02662321F048
:105A80008EE070E00E947821C0E050E08091AA0290
:105A9000882339F4552329F48EE060E070E00E94F9
:105AA00078218091AA02882339F0CC2329F08EE056
:105AB0006C2F70E00E947821CF9108952F923F9231
:105AC0004F925F926F927F928F929F92AF92BF920E
:105AD000CF92DF92EF92FF920F931F93DF93CF93BA
:105AE000CDB7DEB7C555D0400FB6F894DEBF0FBEB8
:105AF000CDBF2C013B011A013AA329A39E2CAF2C48
:105B0000802EB12EDCAACBAA80914C0A41DB649690
:105B10008FAF6497082F112707FD109505C00E94CD
:105B2000AB4381E00E946C1080914D0A90E0801799
:105B30009107A9F3D2016D917D918D919C91209156
:105B400020053091210540912205509123050E94A6
:105B500012520E94E2516FAB78AF89AF9AAFF30156
:105B60006081718182819381209124053091250586
:105B700040912605509127050E9412520E94E25141
:105B80006BAF7CAF8DAF9EAFD1016D917D918D914B
:105B90009C91209128053091290540912A0550912A
:105BA0002B050E9412520E94E2516FAF21967FAFE7
:105BB000219722968FAF229723969FAF2397E9A133
:105BC000FAA1608171818281938120912C053091AD
:105BD0002D0540912E0550912F050E9412520E94D2
:105BE000E2516FA778AB89AB9AAB80917805909121
:105BF0007905A0917A05B0917B052FA538A949A90F
:105C00005AA9281739074A075B0709F445C060916C
:105C1000A902E62FF0E0EE0FFF1FE355F54F80815C
:105C200091810E94A64220E030E046E153E40E94C8
:105C30003D4F87FF31C080914E0A882369F54FA5FB
:105C400058A969A97AA9409378055093790560937A
:105C50007A0570937B05EEE4F4E007C09091C000F4
:105C600095FFFCCF8093C600319684918823B1F7CD
:105C7000E2E7F4E007C09091C00095FFFCCF80936D
:105C8000C600319684918823B1F78091C00085FFCA
:105C9000FCCF8AE08093C6008091780590917905C9
:105CA000A0917A05B0917B052FA538A949A95AA9D9
:105CB000281B390B4A0B5B0BCA01B90157FF07C000
:105CC00090958095709561957F4F8F4F9F4F0E9463
:105CD000DF4F7B018C0160912C0570912D05809127
:105CE0002E0590912F0520E030E04DEC53E40E940A
:105CF00012529B01AC01C801B7010E944051181615
:105D00006CF54FA558A969A97AA9409378055093D5
:105D1000790560937A0570937B05EEE4F4E007C0A3
:105D20009091C00095FFFCCF8093C600319684917E
:105D30008823B1F7E4E5F4E007C09091C00095FF37
:105D4000FCCF8093C600319684918823B1F780916F
:105D5000C00085FFFCCF8AE08093C60080914C0A8A
:105D6000682F70E07AA369A38DE490E0689FF0014A
:105D7000699FF00D789FF00D1124E458FA4FDF0170
:105D8000A45BBF4F1C9280916C0590916D05A09112
:105D90006E05B0916F058BA39CA3ADA3BEA38FA985
:105DA00098ADA9ADBAAD2BA13CA14DA15EA1821BBE
:105DB000930BA40BB50BB7FF07C0B095A0959095BA
:105DC00081959F4FAF4FBF4F80839183A283B38351
:105DD0004091700550917105609172057091730545
:105DE0004FA358A769A77AA78DE490E069A17AA18B
:105DF000689FF001699FF00D789FF00D1124E45821
:105E0000FA4F8BAD9CADADADBEAD2FA138A549A568
:105E10005AA5821B930BA40BB50BB7FF07C0B09517
:105E2000A095909581959F4FAF4FBF4F84839583E9
:105E3000A683B783409174055091750560917605EE
:105E4000709177054BA75CA76DA77EA78DE490E0C6
:105E500069A17AA1689FF001699FF00D789FF00D0C
:105E60001124E458FA4F23968CAD9DADAEADBFAD75
:105E700023972BA53CA54DA55EA5821B930BA40BD8
:105E8000B50BB7FF07C0B095A095909581959F4F32
:105E9000AF4FBF4F80879187A287B3874090780527
:105EA0005090790560907A0570907B052091EC0107
:105EB0003091ED016FA578A989A99AA9641975098E
:105EC0008609970997FF07C0909580957095619511
:105ED0007F4F8F4F9F4F442737FD4095542F0E948F
:105EE000D85224E630E040E050E00E942C538DE48C
:105EF00090E069A17AA1689FF001699FF00D789FF9
:105F0000F00D1124E458FA4F2487358746875787C8
:105F1000C080D18072816381E480F5800681178121
:105F200080859185A285B3858E159F05A007B10751
:105F300014F4D801C70182179307A407B50714F416
:105F4000DA01C901FB0196014F2F562F2817390797
:105F50004A075B0714F49C01AD018DE490E0A9A110
:105F6000BAA1A89FF001A99FF00DB89FF00D1124D0
:105F7000E458FA4F208B318B428B538B26303105FE
:105F80004105510510F40C942B399F01285B3F4FBC
:105F90008091AA02482F50E060E070E0D9014D9353
:105FA0005D936D937C93139710A22FA938AD49ADE3
:105FB0005AAD6BA17CA18DA19EA12617370748077A
:105FC000590714F481E080A38BAD9CADADADBEAD9F
:105FD0002FA138A549A55AA582179307A407B5078D
:105FE00084F48DE490E049A15AA1489FF001499FB3
:105FF000F00D589FF00D1124E458FA4F80A18260F3
:1060000080A323966CAD7DAD8EAD9FAD23972BA560
:106010003CA54DA55EA5621773078407950784F418
:106020008DE490E049A15AA1489FF001499FF00DED
:10603000589FF00D1124E458FA4F80A1846080A38A
:106040006FA578A989A99AA964157505860597058C
:1060500084F48DE490E0A9A1BAA1A89FF001A99FC2
:10606000F00DB89FF00D1124E458FA4F80A188601C
:1060700080A38DE490E029A13AA1289FF001299FF7
:10608000F00D389FF00D1124E458FA4FABA9BCA9CC
:106090008C9181A380819181A281B3810097A10518
:1060A000B10509F05A9A8DE490E029A13AA1289F00
:1060B000F001299FF00D389FF00D1124E458FA4F9C
:1060C00084819581A681B7810097A105B10509F06A
:1060D0005A9A8DE490E049A15AA1489FF001499F46
:1060E000F00D589FF00D1124E458FA4F80859185EA
:1060F000A285B3850097A105B10509F05A9A8DE4F0
:1061000090E069A17AA1689FF001699FF00D789FE6
:10611000F00D1124E458FA4F84859585A685B7853E
:106120000097A105B10509F05A9A8DE490E0A9A164
:10613000BAA1A89FF001A99FF00DB89FF00D1124FE
:10614000E458FA4F84859585A685B7850097A10503
:10615000B10549F4F090580510915905E0905A05A1
:1061600000915B0508C0F090400510914105E0905A
:10617000420500914305692D7A2D882D9B2D2F2DE9
:10618000312F4E2D502F0E943D4F87FD04C0F92C1A
:106190001A2DE82C0B2D90914C0A80914D0AE92F75
:1061A000F0E07096E81BF109EF70F070FCA7EBA728
:1061B000BF01882777FD8095982F0E94DF4F4B0104
:1061C0005C0120E030E040E051E40E943D4F87FF59
:1061D00017C02BA53CA52230310594F06F2D712FEF
:1061E0008E2D902FA50194010E94125220E030E0E4
:1061F00040E05EE30E941252F62E172FE82E092F80
:1062000080916C0590916D05A0916E05B0916F0520
:106210002FA938AD49AD5AAD281B390B4A0B5B0B82
:10622000CA01B9010E94DF4F20912005309121055C
:1062300040912205509123050E94444F762E672EEF
:106240008BA39FA3A301382F292F852F942FA32F32
:10625000B22F89839A83AB83BC8380917005909120
:106260007105A0917205B09173052BAD3CAD4DAD9C
:106270005EAD281B390B4A0B5B0BCA01B9010E94AA
:10628000DF4F20912405309125054091260550913E
:1062900027050E94444F2B018BAB24969FAF249778
:1062A000382F292F862F952DA32FB22F8D839E83D4
:1062B000AF83B8878091740590917505A09176059C
:1062C000B091770523962CAD3DAD4EAD5FAD2397D4
:1062D000281B390B4A0B5B0BCA01B9010E94DF4F27
:1062E000209128053091290540912A0550912B05D0
:1062F0000E94444F362E272E28968FAF28972C9633
:106300009FAF2C97A101382F292F852F942FA32FD2
:10631000B22F89879A87AB87BC878090EC019090D9
:10632000ED018091780590917905A0917A05B09161
:106330007B052FA538A949A95AA9281B390B4A0B57
:106340005B0BCA01B9010E94DF4F20912C053091EF
:106350002D0540912E0550912F050E94444F5B0161
:106360006C01B401882777FD8095982F0E94DF4F3C
:106370009B01AC01C601B5010E94125220E030E041
:1063800048EC52E40E94444F6B01B82FA92F4B01F7
:10639000A82EB92E9B01482F592F2D873E874F8756
:1063A000588B8DE490E049A15AA1489FF001499F84
:1063B000F00D589FF00D1124E458FA4F20813181DF
:1063C00042815381211531054105510591F5248103
:1063D000358146815781211531054105510549F522
:1063E00020853185428553852115310541055105AB
:1063F00001F5B6018B2F9A2F20E030E0A9010E9411
:106400004051181624F0B7FAB094B7F8B0948DE460
:1064100090E069A17AA1689FF001699FF00D789FD3
:10642000F00D1124E458FA4F86A697A6A0AAB1AAA7
:1064300047C0A3013BA12FA1652F762D832F922F5B
:106440000E94BD524B015C013BA924962FAD2497BD
:10645000642D752D832F922F0E94BD522B013C017C
:10646000A10128963FAD28972C962FAD2C97652F2C
:10647000722D832F922F0E94BD526BA37CA38DA3FC
:106480009EA3C501B401A30192010E94644E2BA1F9
:106490003CA14DA15EA10E94644E0E947F522DE45A
:1064A00030E0A9A1BAA1A29FF001A39FF00DB29F75
:1064B000F00D1124E458FA4F66A777A780AB91AB93
:1064C0008DE490E0E9A1FAA1E89F6001E99FD00C7A
:1064D000F89FD00C11242CE735E0C20ED31ED60154
:1064E0009E968D909D90AD90BC90D19760E070E0AD
:1064F00080E89FE3A50194010E94444F9B01AC01F9
:106500006F2D712F8E2D902F0E941252362E272E16
:10651000782E692EC501B401D101F3012B2F3A2F3A
:106520004F2F5E2F0E941252F60162A373A384A321
:1065300095A360897189828993890E94DD4FD10179
:10654000F3012B2F3A2F4F2F5E2F0E9412520E94E1
:106550002A4F0E94B14FD601D8966D937D938D93AB
:106560009C93DB978E010F5F1F4FB1E14B2E512C97
:106570004C0E5D1E7201F8016191719181919191B2
:106580008F01D101F3012B2F322D4F2F562D0E9459
:106590001252D7016D937D938D939D937D010415C8
:1065A000150549F7E0E1F5E0F8A7EFA39E012F5D9F
:1065B0003F4F66963FAF2EAF66973F011201DD2435
:1065C000CC24A0E88A2EFFE3BF2ED101ED90FD90F0
:1065D0000D911D911D01AA24A394C801B70120E0CB
:1065E00030E0A9010E94405118162CF0AA24C801DD
:1065F000B701905802C0C801B701D3012D913D9158
:106600004D915D913D012BA33CA34DA35EA30E9440
:106610004051181664F5AA2021F4A801970150589A
:1066200002C0A80197016BA17CA18DA19EA10E942F
:10663000444F9B01AC01ED2DFC2DA82DBB2DBF01BE
:10664000CD010E943D4F87FD12C0AA2021F417FB07
:10665000109517F910956BA17CA18DA19EA1A801A1
:1066600097010E94444FD62EC72E882EB92E6696CB
:10667000EEADFFAD66972E163F0609F0A6CFA60138
:10668000652F7C2D882D9B2D20E030E040E85FE3D6
:106690000E943D4F87FFA8C012015CA24BA2D1010E
:1066A000ED90FD900D911D911D01AA24A394C801A8
:1066B000B70120E030E0A9010E94405118162CF0EB
:1066C000AA24C801B701905802C0C801B701EFA1C0
:1066D000F8A54190519061907190F8A7EFA3A301A4
:1066E00092010E944051181634F5AA2021F4A80105
:1066F0009701505802C0A8019701C301B2010E943E
:10670000444F9B01AC016D2D7C2D882D9B2D0E944B
:106710003D4F87FD10C0AA2021F417FB109517F9F3
:106720001095C301B201A80197010E94444FD62ED3
:10673000C72E882EB92E66962EAD3FAD66972216CF
:10674000330609F0ACCF4BA05CA0D2016D917D91D6
:106750008D919C91D6012B2F3C2D482D5B2D0E94B5
:106760001252F20161937193819391932F01669676
:106770002EAD3FAD6697E217F30739F78DE490E051
:1067800049A15AA1489F8001499F100D589F100DA3
:10679000112404581A4FD80192966D917D918D91D4
:1067A0009C919597D6012B2F3C2D482D5B2D0E9457
:1067B0001252F80162A373A384A395A360AD71ADD7
:1067C00082AD93AD0E94DD4FD6012B2F3C2D482D7D
:1067D0005B2D0E9412520E94B14FD801D8966D9342
:1067E0007D938D939C93DB978DE490E0E9A1FAA1D2
:1067F000E89F8001E99F100DF89F100D11240458A7
:106800001A4FD80150966D917D918D919C9153971F
:106810000E94DD4FF80126A537A540A951A90E9485
:10682000444F562E472E382E292EF8018081918113
:10683000A281B3810097A105B10569F58481958195
:10684000A681B7810097A105B10529F580859185BD
:10685000A285B3850097A105B105E9F4A2019101D4
:10686000652F742F832F922F209148053091490571
:1068700040914A0550914B050E9412520E942A4FA6
:106880000C5B1F4F0E94B14FD8016D937D938D9388
:106890009C93139765C1A2019101652F742D832FDD
:1068A000922D209144053091450540914605509127
:1068B00047050E9412520E942A4F0E94B14F2DE4B8
:1068C00030E0E9A1FAA1E29F8001E39F100DF29F61
:1068D000100D112404581A4FE4E46E2E712C600E32
:1068E000711ED3016D937D938D939C93139780902C
:1068F0005C0590905D05A0905E05B0905F050E94DC
:10690000DD4F6B017C01F80160817181828193818F
:106910000E94DF4F9B01AC01C701B6010E941252D9
:106920006B017C01D80150966D917D918D919C9168
:1069300053970E94DD4F9B01AC01C701B6010E9435
:10694000444F7B018C01C501B4010E94DD4F9B01C6
:10695000AC01C801B7010E94405118162CF4F30194
:1069600080829182A282B3828090600590906105BE
:10697000A0906205B09063058DE490E029A13AA152
:10698000289F8001299F100D389F100D1124045855
:106990001A4F64E4662E712C600E711ED3016D9146
:1069A0007D918D919C910E94DD4F6B017C01F801DE
:1069B00064817581868197810E94DF4F9B01AC01C4
:1069C000C701B6010E9412526B017C01D80150969A
:1069D0006D917D918D919C9153970E94DD4F9B010C
:1069E000AC01C701B6010E94444F7B018C01C50177
:1069F000B4010E94DD4F9B01AC01C801B7010E94A8
:106A0000405118162CF4F30180829182A282B38245
:106A10008090680590906905A0906A05B0906B051C
:106A20008DE490E029A13AA1289F8001299F100DB3
:106A3000389F100D112404581A4F54E4652E712C00
:106A4000600E711ED3016D917D918D919C910E947C
:106A5000DD4F6B017C01F80164857585868597851E
:106A60000E94DF4F9B01AC01C701B6010E94125288
:106A70006B017C01D80150966D917D918D919C9117
:106A800053970E94DD4F9B01AC01C701B6010E94E4
:106A9000444F7B018C01C501B4010E94DD4F9B0175
:106AA000AC01C801B7010E94405118162CF4F30143
:106AB00080829182A282B382809064059090650565
:106AC000A0906605B09067058DE490E029A13AA1F9
:106AD000289F8001299F100D389F100D1124045804
:106AE0001A4F44E4642E712C600E711ED3016D9117
:106AF0007D918D919C910E94DD4F6B017C01F8018D
:106B000060857185828593850E94DF4F9B01AC0172
:106B1000C701B6010E9412526B017C01D801509648
:106B20006D917D918D919C9153970E94DD4F9B01BA
:106B3000AC01C701B6010E94444F7B018C01C50125
:106B4000B4010E94DD4F9B01AC01C801B7010E9456
:106B5000405118162CF4F30180829182A282B382F4
:106B60008DE490E029A13AA1289F8001299F100D72
:106B7000389F100D112404581A4FF801EC5BFF4F99
:106B800060817181828193810E94DD4F6B017C0164
:106B9000D201F1012B2F342D4F2F522D0E94444F43
:106BA000D801D2966D937D938D939C93D597C70111
:106BB000B6012DEB37E346E051E40E9412520E94E9
:106BC000AC4FF801648F758F868F978F20914C059D
:106BD00030914D0540914E0550914F052B962CAFAD
:106BE0003DAF4EAF5FAF2B97498D5A8D6B8D7C8D2E
:106BF0004BAB5CAB6DAB7EABCB01BA0120E030E0C0
:106C0000A9010E94405118164CF08BA89CA8ADA871
:106C1000BEA8B7FAB094B7F8B09404C08BA89CA8EB
:106C2000ADA8BEA8609150057091510580915205A4
:106C3000909153052F966CAF7DAF8EAF9FAF2F977E
:106C400020E030E040E05FE30E9412527B016C01E3
:106C5000C501B4012E2D3F2D4C2D5D2D0E944051BC
:106C6000181674F02B966CAD7DAD8EAD9FAD2B9745
:106C700020E030E040E05FE30E9412527B016C01B3
:106C80008DE490E0E9A1FAA1E89FD001E99FB00D61
:106C9000F89FB00D1124A458BA4FFD01B2969296F8
:106CA0003C90218022812BA333813FA36E2D7F2D29
:106CB0008C2D9D2DD101FBA1EFA12B2F3A2F4F2F12
:106CC0005E2F0E943D4F87FD04C0E32CF22CCBA029
:106CD000DFA04D8D5E8D6F8D78A127964CAF5DAF97
:106CE0006EAF7FAF2797CB01BA0120E030E0A9015A
:106CF0000E94405118165CF027968CAC9DACAEAC4F
:106D0000BFAC2797B7FAB094B7F8B09406C02796EF
:106D10008CAC9DACAEACBFAC279760915405709124
:106D20005505809156059091570563966CAF7DAFE0
:106D30008EAF9FAF639720E030E040E05FE30E94BA
:106D40001252162F072F482E792EC501B401D801F3
:106D50002B2F3A2F442D572D0E94405118168CF49A
:106D60006E2D7F2D8C2D9D2DD8012B2F3A2F442D4C
:106D7000572D0E943D4F87FD04C0E12EF02EC42CFC
:106D8000D72C8BA59CA5823091050CF469C160912C
:106D90004F0A7091500A8091510A9091520A27E14E
:106DA00037EB41ED58E30E94405118160CF058C1E2
:106DB0002091530A3091540A4091550A5091560A35
:106DC0002BA73CA74DA75EA769897A898B899C89E7
:106DD0000E94634E9B01AC010E941252162F072F96
:106DE000782E692E8090570A9090580AA090590AE0
:106DF000B0905A0A6D897E898F89988DA50194017A
:106E00000E94634E9B01AC010E941252B62FA72F25
:106E1000F82FE92FB801C301272F362F492F582FFC
:106E2000CA01B9018D013F01212F302F472D562D69
:106E30000E94644E0E947F522B013C016BA57CA5F1
:106E40008DA59EA520E030E0A9010E9440511816B2
:106E50006CF46BA57CA58DA59EA527E137EB41EDD4
:106E600058E30E94405118167CF10CC06BA57CA51C
:106E70008DA59EA527E137EB41ED58EB0E943D4FD4
:106E800087FD22C0C501B40120E030E0A9010E94C5
:106E9000405118165CF4C501B40127E137EB41ED10
:106EA00058E30E94405118167CF00AC0C501B40195
:106EB00027E137EB41ED58EB0E943D4F87FD04C0C1
:106EC0003E2C2F2CCBA2DFA2C301B2012B962CADFE
:106ED0003DAD4EAD5FAD2B970E9440511816CCF4DE
:106EE0002B966CAD7DAD8EAD9FAD2B97A30192011E
:106EF0000E94444F9B01AC01D101FBA1EFA16B2F7C
:106F0000722D8F2F9E2F0E941252362E272E8BA36A
:106F10009FA36BA97CA98DA99EA920915B0A3091A2
:106F20005C0A40915D0A50915E0A0E94634ED62E23
:106F3000C72EB82E892EE62EF72E082F192FAA2439
:106F4000A39420E030E0A9010E94405118162CF0D3
:106F5000AA24C801B701905804C06D2D7C2D8B2D3B
:106F6000982D2F962CAD3DAD4EAD5FAD2F970E9465
:106F700040511816FCF4AA2021F417FB109517F9BC
:106F800010952F966CAD7DAD8EAD9FAD2F97A8015E
:106F900097010E94444F9B01AC01D101FBA1EFA1DD
:106FA0006B2F722D8F2F9E2F0E941252362E272E5E
:106FB0008BA39FA327966CAD7DAD8EAD9FAD27971C
:106FC00020915F0A3091600A4091610A5091620AF3
:106FD0000E94634ED62EC72EB82E892EE62EF72E8F
:106FE000082F192FAA24A39420E030E0A9010E94C1
:106FF000405118162CF0AA24C801B701905804C0BB
:107000006D2D7C2D8B2D982D63962CAD3DAD4EAD09
:107010005FAD63970E9440511816F4F4AA2021F442
:1070200017FB109517F9109563966CAD7DAD8EAD7D
:107030009FAD6397A80197010E94444F9B01AC014B
:10704000D101FBA1EFA16B2F722D8F2F9E2F0E94DC
:1070500012527B016C0104C0E32CF22CCBA0DFA008
:107060008DE490E049A15AA1489F8001499F100DED
:10707000589F100D112404581A4F8E2D9F2DAC2DA2
:10708000BD2DF80182A793A7A4A7B5A722A933A96C
:1070900044A955A95058CA01B9010E94644ED801AB
:1070A0009E962D913D914D915C91D1970E941252E7
:1070B0009B01AC016BE077ED83E29BE30E94634EA2
:1070C0000E947F52B62E872EA82E992E6E2D7F2DD0
:1070D0008C2D9D2D2B2D382D4A2D592D0E943D4F45
:1070E00087FD04C0EB2CF82CCA2CD92C8DE490E041
:1070F000E9A1FAA1E89F8001E99F100DF89F100D0A
:10710000112404581A4F8E2D9F2DAC2DBD2DF80142
:1071100086A397A3A0A7B1A762A173A184A195A1FB
:107120002B2D382D4A2D592D0E943D4F181634F025
:1071300081E0D801D7968C93D79702C0F80117AA9F
:107140008DE490E029A13AA1289FF001299FF00D3C
:10715000389FF00D1124E458FA4F81E086ABA3E587
:10716000BAE0FE01719680E101900D928150E1F745
:107170008DE490E049A15AA1489F8001499F100DDC
:10718000589F100D112404581A4FD8019296CD9093
:10719000DD90ED90FC909597C0924F0AD092500AE6
:1071A000E092510AF092520A96966D917D918D91DE
:1071B0009C919997A70196010E94444F4B015C0155
:1071C0006DEC7CEC8CE49DE3A70196010E94444F9A
:1071D0006B017C01C801B501A401970186010E94E1
:1071E000CD286496BFAD6497B0934C0A2FA938ADF3
:1071F00049AD5AAD20936C0530936D0540936E05F3
:1072000050936F054BAD5CAD6DAD7EAD4093700599
:1072100050937105609372057093730523966CAD5E
:107220007DAD8EAD9FAD239760937405709375050A
:1072300080937605909377058FA598A9A9A9BAA9F7
:107240008093780590937905A0937A05B0937B0598
:107250000E94CC2CACD1CB5ADF4F0FB6F894DEBFD6
:107260000FBECDBFCF91DF911F910F91FF90EF9097
:10727000DF90CF90BF90AF909F908F907F906F9056
:107280005F904F903F902F900895CF92DF92EF92B2
:10729000FF920F931F93CF93DF938B017A016901C4
:1072A000FC01608171818281938120912005309160
:1072B000210540912205509123050E9412520E94FF
:1072C000E251CCE6D5E060936C0570936D05809338
:1072D0006E0590936F05F8016081718182819381C1
:1072E00020912405309125054091260550912705D0
:1072F0000E9412520E94E2518E010C5F1F4F609358
:107300007005F801718382839383F7016081718135
:1073100082819381209128053091290540912A0589
:1073200050912B050E9412520E94E25128E0E22E59
:10733000F12CEC0EFD1E60937405F70171838283BE
:107340009383F601608171818281938120912C0564
:1073500030912D0540912E0550912F050E9412521B
:107360000E94E251FE013C9660937805718382830E
:107370009383CE01B801A7019F0160D780E090E020
:10738000DC0180934F0A9093500AA093510AB09366
:10739000520A8093530A9093540AA093550AB093CB
:1073A000560A8093570A9093580AA093590AB093AB
:1073B0005A0A80935B0A90935C0AA0935D0AB0938B
:1073C0005E0A80935F0A9093600AA093610AB0936B
:1073D000620ADF91CF911F910F91FF90EF90DF90A4
:1073E000CF900895FC016081718182819381209109
:1073F0002C0530912D0540912E0550912F050E94AE
:1074000012520E94E251609378057093790580933F
:107410007A0590937B0588E795E04CC780934E0AE8
:1074200008958091970A882349F48091990A8823C6
:1074300029F480919B0A882309F4AEC0ECE8FCE0B3
:1074400007C09091C00095FFFCCF8093C600319695
:1074500084918823B1F7EEE9FCE007C09091C00069
:1074600095FFFCCF8093C600319684918823B1F7B5
:107470008091970A882349F1EAE9FCE007C09091DE
:10748000C00095FFFCCF8093C6003196849188237D
:10749000B1F76091650A7091660A8091670A9091D0
:1074A000680A0E94DF4F209120053091210540910C
:1074B0002205509123050E94444FAB01BC018BE093
:1074C00095E022E030E00E9475248091990A88239B
:1074D00049F1E6E9FCE007C09091C00095FFFCCFC0
:1074E0008093C600319684918823B1F76091690A30
:1074F00070916A0A80916B0A90916C0A0E94DF4F2A
:1075000020912405309125054091260550912705AD
:107510000E94444FAB01BC018BE095E022E030E0DB
:107520000E94752480919B0A882349F1E2E9FCE0DE
:1075300007C09091C00095FFFCCF8093C6003196A4
:1075400084918823B1F760916D0A70916E0A8091E1
:107550006F0A9091700A0E94DF4F209128053091A8
:10756000290540912A0550912B050E94444FAB01FB
:10757000BC018BE095E022E030E00E947524809110
:10758000C00085FFFCCF8AE08093C6001092970A66
:107590001092990A10929B0A08951092970A1092DD
:1075A000990A10929B0A08958093FB010895EFE6D3
:1075B000F0E080818260808308951F920F920FB661
:1075C0000F9211242F923F924F925F926F927F926F
:1075D0008F929F92AF92BF92CF92DF92EF92FF92E3
:1075E0000F931F932F933F934F935F936F937F93CB
:1075F0008F939F93AF93BF93EF93FF93DF93CF93BB
:1076000000D000D0CDB7DEB78091630A9091640AB4
:10761000009709F05DC190914C0A80914D0A98172E
:10762000A1F020914D0A30E08DE490E0289FF00118
:10763000299FF00D389FF00D1124E458FA4FDF0117
:10764000A45BBF4F81E08C9302C0E0E0F0E0F093D8
:10765000640AE093630A309709F434C11092A30AD4
:107660001092A40A1092A50A1092A60A34AD25AD74
:107670003093A10A2093A20AC901692F782F27E22B
:107680006131720710F060E177E281E080939C0A3B
:107690006832710510F468E270E06852704038E0BA
:1076A00060307307E0F0872F90E0880F991F880FF4
:1076B000991F84579B4FFC01329645915491AA27FC
:1076C000659F9001649F210D3A1F06942A1F3A1F5F
:1076D0001124FC0145915491421B530B1FC0CB0157
:1076E000969587958C7F8457974FFC0145915491CF
:1076F0000296FC0125913491E62FF0E0E770F070DE
:107700002E9FC0012F9F900D3E9F900D1124E3E00E
:1077100096958795EA95E1F7481B590B4436510534
:10772000A0F4E3EBF1E006C09091C00095FFFCCF20
:107730008093C60081918823B9F78BE095E04AE0F9
:1077400050E00E94B92344E650E0CA01A0E0B0E056
:1077500080939D0A90939E0AA0939F0AB093A00ADB
:107760005093890040938800E091630AF091640A85
:1077700090AD81AD692F782F87E26131780710F0E5
:1077800060E177E281E080939C0A6832710510F431
:1077900068E270E068527040E8E060307E07E0F038
:1077A000872F90E0880F991F880F991F84579B4F50
:1077B000FC01329645915491AA27659F9001649FE0
:1077C000210D3A1F06942A1F3A1F1124FC014591EE
:1077D0005491421B530B1FC0CB01969587958C7F0C
:1077E0008457974FFC01459154910296FC012591D5
:1077F0003491E62FF0E0E770F0702E9FC0012F9FCC
:10780000900D3E9F900D112403E0969587950A9563
:10781000E1F7481B590B44365105A0F4E3EBF1E0C6
:1078200006C09091C00095FFFCCF8093C600819167
:107830008823B9F78BE095E04AE050E00E94B92335
:1078400044E650E05093A80A4093A70AE091630AE7
:10785000F091640A80899189A289B389B695A79528
:1078600097958795B095A095909581959F4FAF4F2F
:10787000BF4F8093810A9093820AA093830AB093AA
:10788000840A8093850A9093860AA093870AB0930E
:10789000880A8093890A90938A0AA0938B0AB093EE
:1078A0008C0A80938D0A90938E0AA0938F0AB093CE
:1078B000900A1092910A1092920A1092930A1092D2
:1078C000940A06C080ED97E0909389008093880029
:1078D000E091630AF091640A309709F43EC480A1F4
:1078E0008093950A80FF37C016988FEF8093F70139
:1078F00023B1217031E0232759F18091960A882322
:1079000039F180819181A281B381181619061A0676
:107910001B06F4F48091710A9091720AA091730A87
:10792000B091740A8093650A9093660AA093670ADF
:10793000B093680A3093970A80899189A289B389A4
:107940008093910A9093920AA093930AB093940A19
:107950002093960A04C0169A81E08093F7018091E3
:10796000950A81FF3BC0149A8FEF8093F80121E0C4
:10797000199B02C020E02FC08091980A882359F1FA
:10798000E091630AF091640A84819581A681B781B0
:10799000181619061A061B06F4F48091750A9091C0
:1079A000760AA091770AB091780A8093690A909339
:1079B0006A0AA0936B0AB0936C0A2093990A808993
:1079C0009189A289B3898093910A9093920AA09396
:1079D000930AB093940A2093980A04C0149881E003
:1079E0008093F8018091950A82FF3BC046988FEF03
:1079F0008093F90121E01A9B02C020E02FC0809102
:107A00009A0A882359F1E091630AF091640A80850B
:107A10009185A285B385181619061A061B06F4F47B
:107A20008091790A90917A0AA0917B0AB0917C0AA0
:107A300080936D0A90936E0AA0936F0AB093700AB8
:107A400020939B0A80899189A289B3898093910AA6
:107A50009093920AA093930AB093940A20939A0A5F
:107A600004C0469A81E08093F9018091950A83FFD2
:107A700003C045988FEF02C0459A81E08093FA01D8
:107A800080919C0A282F30E03A8329832091810A33
:107A90003091820A4091830A5091840A8091850A2C
:107AA0009091860AA091870AB091880AA090890ACD
:107AB000B0908A0AC0908B0AD0908C0A60908D0A90
:107AC00070908E0A80908F0A9090900A1C821B8280
:107AD00035C16091C00067FF19C02090C600E091D9
:107AE0000705F0910805BF016F5F7F4F6F777070DA
:107AF000E0900905F0900A056E157F0539F0E95709
:107B0000FB4F20827093080560930705E091630A9C
:107B1000F091640AE080F180028113812E0D3F1DF7
:107B2000401F511F12161306140615060CF4159A61
:107B3000E091630AF091640AE480F5800681178180
:107B40008E0D9F1DA01FB11F181619061A061B06C1
:107B50000CF4139AE091630AF091640AE084F184D2
:107B600002851385AE0CBF1CC01ED11E1A141B0447
:107B70001C041D040CF4479AE091630AF091640A16
:107B8000E484F584068517856E0C7F1C801E911E8B
:107B900016141704180419040CF4179A1216130675
:107BA000140615061CF5E091630AF091640AE0885A
:107BB000F188028913892E193F09400B510BE0907F
:107BC000710AF090720A0091730A1091740A609120
:107BD000F701E60EF11C011D111DE092710AF092F1
:107BE000720A0093730A1093740A159818161906EE
:107BF0001A061B061CF5E091630AF091640AE088FE
:107C0000F188028913898E199F09A00BB10BE090AE
:107C1000750AF090760A0091770A1091780A6091BF
:107C2000F801E60EF11C011D111DE092750AF0929B
:107C3000760A0093770A1093780A13981A141B0493
:107C40001C041D041CF5E091630AF091640AE088AD
:107C5000F18802891389AE18BF08C00AD10AE090E2
:107C6000790AF0907A0A00917B0A10917C0A60915F
:107C7000F901E60EF11C011D111DE092790AF09246
:107C80007A0A00937B0A10937C0A4798161417040B
:107C9000180419041CF5E091630AF091640AE08865
:107CA000F188028913896E187F08800A910AE09092
:107CB0007D0AF0907E0A00917F0A1091800A6091FF
:107CC000FA01E60EF11C011D111DE0927D0AF092F1
:107CD0007E0A00937F0A1093800A1798E090910A19
:107CE000F090920A0091930A1091940A0894E11C72
:107CF000F11C011D111DE092910AF092920A00936D
:107D0000930A1093940A2090910A3090920A40901E
:107D1000930A5090940A6B817C816F5F7F4F7C83C4
:107D20006B83E091630AF091640AE088F18802892C
:107D300013892E143F044006510640F4EB81FC8168
:107D400069817A81E617F7070CF4C3CE2093810A84
:107D50003093820A4093830A5093840A8093850A61
:107D60009093860AA093870AB093880AA092890A02
:107D7000B0928A0AC0928B0AD0928C0A60928D0AC5
:107D800070928E0A80928F0A9092900A2091910AA6
:107D90003091920A4091930A5091940AE091630ABB
:107DA000F091640A84899589A689B7898217930717
:107DB000A407B50708F4C8C020919D0A30919E0A17
:107DC00040919F0A5091A00A648D758D868D978D84
:107DD000AA27279FB12D389F7001489FF00C479F1D
:107DE000E00CF11C289FB00DE11CFA1E379FB00D6E
:107DF000E11CFA1E469FB00DE11CFA1E369FB10D24
:107E0000EA1EFA1EB695EA1EFA1E112424AD35ADFF
:107E10002E0D3F1D3093A20A2093A10A80AD91AD93
:107E2000A2ADB3AD40E050E082179307A407B507B9
:107E300020F49093A20A8093A10A9091A10A8091C4
:107E4000A20A692F782F87E26131780710F060E18C
:107E500077E281E080939C0A6832710510F468E251
:107E600070E068527040E8E060307E07E0F0872FF5
:107E700090E0880F991F880F991F84579B4FFC0132
:107E8000329625913491AA27639FA001629F410DEC
:107E90005A1F06944A1F5A1F1124FC012591349140
:107EA000241B350B1FC0CB01969587958C7F84577B
:107EB000974FFC01259134910296FC014591549114
:107EC000E62FF0E0E770F0704E9FC0014F9F900DDD
:107ED0005E9F900D1124F3E096958795FA95E1F752
:107EE000281B390B24363105A0F4E3EBF1E006C082
:107EF0009091C00095FFFCCF8093C60081918823AC
:107F0000B9F78BE095E04AE050E00E94B92324E6FF
:107F100030E0309389002093880040E050E0809169
:107F20009D0A90919E0AA0919F0AB091A00A820F8B
:107F3000931FA41FB51F80939D0A90939E0AA09340
:107F40009F0AB093A00AE4C02091910A3091920A4E
:107F50004091930A5091940A808D918DA28DB38D9A
:107F600082179307A407B50708F0CAC02091A30A97
:107F70003091A40A4091A50A5091A60A648D758D8E
:107F8000868D978DAA27279FB12D389F7001489F16
:107F9000F00C479FE00CF11C289FB00DE11CFA1E6D
:107FA000379FB00DE11CFA1E469FB00DE11CFA1E72
:107FB000369FB10DEA1EFA1EB695EA1EFA1E11246E
:107FC0006091A10A7091A20A6E157F0538F4DF0155
:107FD000A05CBF4F6D917C91119702C06E197F0913
:107FE000E05CFF4F80819181A281B3819B0140E0E1
:107FF00050E0281739074A075B0708F4BC01F7E28D
:1080000061317F0710F060E177E281E080939C0AA4
:108010006832710510F468E270E06852704028E040
:1080200060307207E0F0872F90E0880F991F880F6B
:10803000991F84579B4FFC01329625913491AA27B2
:10804000639FA001629F410D5A1F06944A1F5A1F49
:108050001124FC0125913491241B350B1FC0CB0149
:10806000969587958C7F8457974FFC012591349185
:108070000296FC0145915491E62FF0E0E770F07014
:108080004E9FC0014F9F900D5E9F900D112443E0C5
:10809000969587954A95E1F7281B390B24363105CB
:1080A000A0F4E3EBF1E006C09091C00095FFFCCF97
:1080B0008093C60081918823B9F78BE095E04AE070
:1080C00050E00E94B92324E630E0309389002093E9
:1080D000880040E050E08091A30A9091A40AA0910A
:1080E000A50AB091A60A820F931FA41FB51F809303
:1080F000A30A9093A40AA093A50AB093A60A08C065
:108100008091A70A9091A80A909389008093880093
:108110002091910A3091920A4091930A5091940AC9
:10812000E091630AF091640A80899189A289B389F8
:10813000281739074A075B0780F01092640A1092EB
:10814000630A90914C0A80914D0A981731F0809102
:108150004D0A8F5F8F7080934D0A2496DEBFCDBF8E
:10816000CF91DF91FF91EF91BF91AF919F918F914F
:108170007F916F915F914F913F912F911F910F913F
:10818000FF90EF90DF90CF90BF90AF909F908F9037
:108190007F906F905F904F903F902F900F900FBE09
:1081A0000F901F9018950E9A0C9A3E9A3D9A529AEB
:1081B000529A529A529A2098289A2198299A22984B
:1081C0002A9A0D9A0B9A3F9A0F9AA1E8B0E08C91E7
:1081D0008F7E8C938C9188608C93E0E8F0E08081B6
:1081E0008D7F808380818E7F808380818F73808369
:1081F00080818F7C80838C91887F82608C9380E0EB
:1082000090E49093890080938800109285001092EA
:108210008400EFE6F0E080818260808381E0C4D951
:108220007894089590914C0A80914D0A981729F0FE
:1082300092D281E00E946C10F5CF0895CF93DF9326
:10824000EFB7F894EC0188819981AA81BB81809372
:10825000710A9093720AA093730AB093740AEB01A7
:1082600088819981AA81BB818093750A9093760A4F
:10827000A093770AB093780AEA0188819981AA814C
:10828000BB818093790A90937A0AA0937B0AB0937A
:108290007C0AE90188819981AA81BB8180937D0A4A
:1082A00090937E0AA0937F0AB093800AEFBFDF917C
:1082B000CF9108952FB7F894FC0180819181A2811C
:1082C000B38180937D0A90937E0AA0937F0AB09336
:1082D000800A2FBF08959FB7F894E82FF0E0EE0FC3
:1082E000FF1FEE0FFF1FEF58F54F208131814281B4
:1082F00053819FBFB901CA01089594DF5A985A98D3
:108300005A985A98089560E070E08FE793E42091BE
:1083100000023091010240910202509103020E943A
:10832000444F6093D00A7093D10A8093D20A9093FD
:10833000D30A0895FC01EB54F54F808190E0089535
:108340000F931F93CF93DF93EC01062F662359F110
:10835000EDEAFCE007C09091C00095FFFCCF809350
:10836000C600319684918823B1F78BE095E0602FA9
:1083700070E04AE050E00E949C23E9E5FEE007C07F
:108380009091C00095FFFCCF8093C60031968491F8
:108390008823B1F78091C00085FFFCCF8AE08093ED
:1083A000C6000E944310602F70E0660F771FFB012C
:1083B000EF57FD4F80819181009709F45BC06D57A5
:1083C0007D4FFB01A081B18101E037C0A901440FBD
:1083D000551F440F551FFA013296E80FF91F65919A
:1083E00074916C177D0744F5D9011197AA0FBB1F33
:1083F000AA0FBB1FFC01EA0FFB1F259134911296B7
:10840000A80FB91FFD0105911491840F951FFC0160
:10841000A591B491A21BB30BC01BD10BAC9FC001A3
:10842000AD9F900DBC9F900D1124601B710B0E949D
:10843000F752620F731F19C00F5F202F30E02A1709
:108440003B070CF4C3CF2A173B0769F41197AA0F17
:10845000BB1FAA0FBB1FA80FB91FFD0185919491E7
:10846000682F792F02C060E070E020EF3FE3261B09
:10847000370B16C0BE01882777FD8095982F0E9484
:10848000DF4F2FE632E143E050E40E94125220E039
:1084900030E040E851E40E9412520E94AC4F9B0130
:1084A000C901DF91CF911F910F91089520E030E035
:1084B000D9011196AD01440F551F440F551FFA0104
:1084C000E65BF24F65917491681779073CF5D90125
:1084D000AA0FBB1FAA0FBB1FFD01E85BF24F25913E
:1084E0003491A65BB24FFD01A591B491485B524F08
:1084F000FA0145915491421B530BFC01EA1BFB0B03
:108500004E9FC0014F9F900D5E9F900D11246A1BDE
:108510007B0B0E94F752620F731F12C0422F4E5FF7
:108520009D01AC33B10509F0C3CF4D3339F4E8E315
:10853000FEE085919491682F792F02C060E070E091
:1085400020EF3FE3261B370BC90108952F923F927E
:108550004F925F926F927F928F929F92AF92BF9253
:10856000CF92DF92EF92FF920F931F93CF93DF93FF
:108570008C01C62F662359F1EDEAFCE007C090910B
:10858000C00095FFFCCF8093C6003196849188236C
:10859000B1F78BE095E06C2F70E04AE050E00E946C
:1085A0009C23ECE3FEE007C09091C00095FFFCCF58
:1085B0008093C600319684918823B1F78091C000E2
:1085C00085FFFCCF8AE08093C6000E9443106C2F89
:1085D00070E0660F771FFB01EF57FD4F808191819F
:1085E000009709F488C0C0EFDFE3C01BD10B6D57C3
:1085F0007D4FFB0160817181A1E060C09A01220F73
:10860000331F220F331FFC01E20FF31FA590B4901C
:10861000CA15DB050CF051C041505040440F551FA6
:10862000440F551FFA013296E80FF91F0591149176
:10863000480F591FFA01859094902E5F3F4F280FE5
:10864000391FF90165907490B801882777FD8095EE
:10865000982F0E94DF4F1B012C01C819D909BE01B8
:10866000882777FD8095982F0E94DF4F6B017C0152
:10867000601A710AB301882777FD8095982F0E94B0
:10868000DF4F9B01AC01C701B6010E9412527B0172
:108690008C01A818B908B501882777FD8095982F17
:1086A0000E94DF4F9B01AC01C801B7010E94444FFB
:1086B0009B01AC01C201B10134C0AF5F4A2F50E051
:1086C000461757070CF49ACF4617570769F5660FF8
:1086D000771F660F771F62507040680F791FFB018C
:1086E000859194919C01B901882777FD8095982FF9
:1086F0000E94DF4F1DC0B801882777FD8095982F15
:108700000E94DF4F20E030E04AEF5EE30E94125209
:1087100020E030E040E85DE30E94125220E030E0CB
:10872000A9010E94644E04C060E070E080E090E027
:10873000DF91CF911F910F91FF90EF90DF90CF903D
:10874000BF90AF909F908F907F906F905F904F9071
:108750003F902F9008954F925F926F927F928F92E9
:108760009F92AF92BF92CF92DF92EF92FF920F93C0
:108770001F93CF93DF938091B60A882309F4C7C172
:108780008FB7F8941092B60A8FBF8091AD0A90917E
:10879000AE0A60E0DBDE4B015C016091B10A7091D2
:1087A000B20A8091B30A9091B40AA50194010E9483
:1087B000634EEB01182F092F9801862F9D2FA32FB1
:1087C000B22F8093D40A9093D50AA093D60AB0937F
:1087D000D70A6C2F7D2F832F922F20E030E040E2CC
:1087E00051E40E94405118160CF42DC198016C2FD1
:1087F0007D2F832F922F20E030E040E251EC0E9449
:108800003D4F87FD1CC18091D80A882309F009C11A
:1088100098016C2F7D2F832F902F2091FC01309198
:10882000FD014091FE015091FF010E9412522B0167
:108830003C01862F952DA62DB72D8093DD0A9093B0
:10884000DE0AA093DF0AB093E00A98016C2F7D2F17
:10885000832F902F2091D90A3091DA0A4091DB0AB8
:108860005091DC0A0E94644EF62EE72ED82EC92EB7
:108870000091CC0A1091CD0AD091CE0AC091CF0AB6
:10888000A7019601652F742F832F922FFE01202FB1
:10889000312F4F2F5E2F0E943D4F87FFA6C09E01B4
:1088A000802F912FA32FBC2F8093D90A9093DA0A9F
:1088B000A093DB0AB093DC0A602F712F832F9C2FCB
:1088C0002091000230910102409102025091030276
:1088D0000E941252D62FC72F182F092FAE019801D0
:1088E000852F942FA32FB22F8093E10A9093E20A51
:1088F000A093E30AB093E40AC501B4012091E50A0C
:108900003091E60A4091E70A5091E80A0E94634ECE
:108910002091040230910502409106025091070215
:108920000E94125220ED3CEC4CE45DE30E94125296
:108930006B017C016091E90A7091EA0A8091EB0A6F
:108940009091EC0A23E333E343E75FE30E94125282
:108950009B01AC01C701B6010E94644E7B01D82E79
:10896000C92E9601862F9F2DA32FB22F8093E90A3F
:108970009093EA0AA093EB0AB093EC0A8092E50A7E
:108980009092E60AA092E70AB092E80A642D752D4B
:10899000862D972DDE01F8012B2F3A2F4F2F5E2FBA
:1089A0000E94644EF6012E2D3F2D4F2F5E2F0E9408
:1089B000634E8B01D82FC92F9E01712F832F922FC9
:1089C00020E030E0A9010E943D4F87FD44C09E0198
:1089D000602F712F832F922F20E030E04FE753E478
:1089E0000E9440511816DCF531C00091D00A109158
:1089F000D10AD091D20AC091D30AA7019601652F5E
:108A0000742F832F922FFE01202F312F4F2F5E2F97
:108A10000E94405118160CF442CF0F2D1E2DE60176
:108A20003ECF80E090E0DC018093D90A9093DA0A8F
:108A3000A093DB0AB093DC0A1092D80AE9CE81E059
:108A40008093D80A08C081E08093D80A00E010E043
:108A5000DFE7C3E404C000E010E0D0E0C0E08091B4
:108A6000AD0A9091AE0A2091B70A3091B80A281742
:108A700039071CF01092B50A12C020910C023091F7
:108A80000D0282179307B4F79E01602F712F832F79
:108A90009C2F0E94AC4F759567956093B50A0E9414
:108AA000E2202091ED0A3091EE0A4091EF0A5091B8
:108AB000F00A621B730B840B950B683823E1720775
:108AC00020E0820720E0920710F10E94E2206093EC
:108AD000ED0A7093EE0A8093EF0A9093F00A80916A
:108AE000AF0A9091B00A1816190684F420910E026C
:108AF00030910F02821793074CF42091AB0A30910A
:108B0000AC0A8217930714F42C9A01C02C98DF91B9
:108B1000CF911F910F91FF90EF90DF90CF90BF907A
:108B2000AF909F908F907F906F905F904F9008953F
:108B30002F923F924F925F926F927F928F929F926D
:108B4000AF92BF92CF92DF92EF92FF920F931F935B
:108B5000DF93CF93CDB7DEB7E9970FB6F894DEBFBA
:108B60000FBECDBF6D877E878F87988B8FE78093F1
:108B7000B50A0E94E2206B8B7C8B8D8B9E8BE7EC81
:108B8000F1E006C09091C00095FFFCCF8093C60035
:108B900081918823B9F78091C00085FFFCCF8AE0DE
:108BA0008093C6002B893C894D895E892B8F3C8F31
:108BB0004D8F5E8F2F8B388F498F5A8F8FE790E0C4
:108BC000A0E0B0E089839A83AB83BC833FE7432E68
:108BD000512C612C712C11E01A8A198AECE2FFE009
:108BE00094919CA7E7E2FFE0A491ADA7E0E2FFE04B
:108BF000B491BEA7E9E1FFE024912FA7E3E1FFE0F4
:108C0000349138ABEDE0FFE0449149ABE0E0FFE0A8
:108C100054915AABEAEFFEE084918BABE4EFFEE0B7
:108C200094919CABEEEEFEE0A491ADABEDEDFEE0D9
:108C3000B491BEABE7EDFEE024912FAB8091B60A74
:108C4000882309F461C48FB7F8941092B60A8FBFD5
:108C50008091AD0A9091AE0A60E078DC6D837E83EE
:108C60008F8398875F8D48A139A12AA1652F742F22
:108C7000832F922FBD81AE81DF80C8842B2F3A2FA6
:108C80004D2D5C2D0E944051181634F03D813F8FD0
:108C90004E8148A3D9A2CAA26F2D702F8E2D992D77
:108CA000BD81AE81DF80C8842B2F3A2F4D2D5C2DE6
:108CB0000E943D4F87FD04C0FD800E81ED2C9C2C51
:108CC000112309F454C05D814E813F812885652FB1
:108CD000742F832F922FBD85AE85DF84C8882B2FFC
:108CE0003A2F4D2D5C2D0E94405118160CF00CC4EB
:108CF0000E94E2202B8D3C8D4D8D5E8D621B730B8F
:108D0000840B950B693833E1730730E0830730E05B
:108D1000930708F4F9C3D301C20129813A814B8139
:108D20005C81821B930BA40BB50BB595A79597950A
:108D300087958093B50A0E94E2206F8B788F898F88
:108D40009A8FDC01CB012B8D3C8D4D8D5E8D821B6E
:108D5000930BA40BB50B88A799A7AAA7BBA73D8522
:108D60003F8F4E8548A35F8559A388898AA35D817B
:108D70004E813F812885652F742F832F922FBD85CB
:108D8000AE851F85D8882B2F3A2F412F5D2D0E944D
:108D90003D4F87FFB8C30E94E2202F89388D498D4F
:108DA0005A8D621B730B840B950B693833E1730783
:108DB00030E0830730E0930708F4A5C30E94E22067
:108DC0006B8F7C8F8D8F9E8F49895A8941155105F4
:108DD00009F47FC3DC01CB012F89388D498D5A8D71
:108DE000821B930BA40BB50B28A539A54AA55BA53F
:108DF000280F391F4A1F5B1F29873A874B875C87DB
:108E000028A539A54AA55BA5281B390B4A0B5B0B86
:108E1000CA01B90129813A814B815C810E94D852F3
:108E200029853A854B855C850E942C53240D351D80
:108E3000461D571D243131054105510504F1290115
:108E40003A013CEE43165104610471042CF09BEE90
:108E5000492E512C612C712C40E8441651046104B8
:108E60007104DCF08EEF90E0A0E0B0E08419950989
:108E7000A609B70989839A83AB83BC8312C084E1B6
:108E8000482E512C612C712C24E130E040E050E060
:108E900029833A834B835C8304C049825A826B8264
:108EA0007C828CA5ECE2FFE008C09091C00095FFA9
:108EB000FCCF8093C600319684918823B1F78BE074
:108EC00095E0B301A2012AE030E00E946C238DA559
:108ED000E7E2FFE008C09091C00095FFFCCF8093CF
:108EE000C600319684918823B1F78BE095E04981E3
:108EF0005A816B817C812AE030E00E946C238EA530
:108F0000E0E2FFE008C09091C00095FFFCCF8093A5
:108F1000C600319684918823B1F78BE095E04F2D00
:108F2000502F6E2D792D22E030E00E9475248FA500
:108F3000E9E1FFE008C09091C00095FFFCCF80936D
:108F4000C600319684918823B1F78BE095E0FF8DC0
:108F5000E8A139A12AA14F2F5E2F632F722F22E0A3
:108F600030E00E9475248091C00085FFFCCF8AE02C
:108F70008093C60049895A89433051050CF4A9C22F
:108F800069817A818B819C810E94DF4F20E030E0F3
:108F900040E850E40E9412525B016C015F8D48A1D1
:108FA00039A12AA1652F742F832F922F2F2D302FB7
:108FB0004E2D592D88D620ED3FE049E450E40E9423
:108FC000125220E030E040E05FE30E9412529B0129
:108FD000AC01C601B50158D76BA37CA38DA39EA39A
:108FE00069857A858B859C85EAD720E030E04AE761
:108FF00054E44AD7F62ED72EC82EB92E88A9E3E11D
:10900000FFE008C09091C00095FFFCCF8093C600A0
:10901000319684918823B1F78BE095E0FBA1ECA118
:109020003DA12EA14F2F5E2F632F722F22E030E043
:109030000E94752489A9EDE0FFE008C09091C0006E
:1090400095FFFCCF8093C600319684918823B1F7B9
:109050008BE095E04F2D5D2D6C2D7B2D22E030E0D7
:109060000E9475248091C00085FFFCCF8AE0809328
:10907000C6005BA14CA13DA12EA1652F742F832FAB
:10908000922F2AE939E949E15FE30E94125269AF60
:1090900078AF182F092F562F472F9801832F922F23
:1090A000DA01F8012B2F3A2F4F2F5E2F0DD62F2DDF
:1090B0003D2D4C2D5B2DE8D6362E272E89879FA37C
:1090C00059AD48AD9801652F742F832F922F2F2D06
:1090D0003D2D4C2D5B2D0E94125220E030E040E0EF
:1090E0005EE30E941252E62EA72E982E892E8AA9A0
:1090F000E0E0FFE039AD98AD0AC0292F9091C000A3
:1091000095FFFCCF922F8093C600319684918823DF
:10911000A1F78091C00085FFFCCF39AF98AF8AE0FE
:109120008093C6008BA9EAEFFEE039AD98AD0AC086
:10913000292F9091C00095FFFCCF922F8093C600FD
:10914000319684918823A1F739AF98AF8BE095E0F1
:10915000F32FE8AD98014F2F5E2F632F702F22E081
:1091600030E00E9475248091C00085FFFCCF8AE02A
:109170008093C6008CA9E4EFFEE008C09091C00087
:1091800095FFFCCF8093C600319684918823B1F778
:109190008BE095E0F10139852FA14F2F522D632FE0
:1091A000722F22E030E00E9475248091C00085FF7C
:1091B000FCCF8AE08093C6008DA9EEEEFEE008C0E9
:1091C0009091C00095FFFCCF8093C60031968491AA
:1091D0008823B1F78BE095E094014E2D5A2D632F33
:1091E000782D22E030E00E9475248091C00085FF38
:1091F000FCCF8AE08093C6005BA14CA13DA12EA1CB
:10920000652F742F832F922F23EC35EF48EA5EE30E
:109210000E94125269AF78AF182F092F9801832F3F
:10922000922F2F2D3D2D4C2D5B2D2ED6362E272EF9
:1092300089879FA359AD48AD9801652F742F832F5F
:10924000922F2F2D3D2D4C2D5B2D0E94125220E090
:1092500030E040E450E418D6E62EA72E982E892E52
:109260008EA9EDEDFEE039AD98AD0AC0292F9091A1
:10927000C00095FFFCCF922F8093C6003196849159
:109280008823A1F78091C00085FFFCCF39AF98AF4C
:109290008AE08093C6008FA9E7EDFEE039AD98AD76
:1092A0000AC0292F9091C00095FFFCCF922F809388
:1092B000C600319684918823A1F739AF98AF8BE02F
:1092C00095E0F32FE8AD98014F2F5E2F632F702F9D
:1092D00022E030E00E9475248091C00085FFFCCF21
:1092E0008AE08093C600E1EDFEE007C09091C000E7
:1092F00095FFFCCF8093C600319684918823B1F707
:109300008BE095E0F10139852FA14F2F522D632F6E
:10931000722F22E030E00E9475248091C00085FF0A
:10932000FCCF8AE08093C600EBECFEE007C0909192
:10933000C00095FFFCCF8093C600319684918823AE
:10934000B1F78BE095E094014E2D5A2D632F782DC7
:1093500022E030E00E9475248091C00085FFFCCFA0
:109360008AE08093C6005BA14CA13DA12EA1652F90
:10937000742F832F922F2DEC3CEC4CE45EE30E9483
:1093800012526987272E182F092F562F9801832FE5
:10939000922FF801252F322D4F2F5E2F95D42F2D90
:1093A0003D2D4C2D5B2D70D5A62E972E882E392E57
:1093B00059859801652F722D832F922F2F2D3D2DCA
:1093C0004C2D5B2D0E94125220E030E040E450E42E
:1093D0005BD5F62EE72ED82EC92EECEBFEE084915D
:1093E00099850AC0292F9091C00095FFFCCF922F3C
:1093F0008093C600319684918823A1F78091C000A4
:1094000085FFFCCF99878AE08093C600E6EBFEE0FB
:10941000849199850AC0292F9091C00095FFFCCFB7
:10942000922F8093C600319684918823A1F7998763
:109430008BE095E0F98598014F2F522D632F702F07
:1094400022E030E00E9475248091C00085FFFCCFAF
:109450008AE08093C600E0EBFEE007C09091C00078
:1094600095FFFCCF8093C600319684918823B1F795
:109470008BE095E04A2D592D682D732D22E030E0C8
:109480000E9475248091C00085FFFCCF8AE0809304
:10949000C600EAEAFEE007C09091C00095FFFCCF4D
:1094A0008093C600319684918823B1F78BE095E0D4
:1094B000F70196014F2F5E2D632F7C2D22E030E0C7
:1094C0000E9475248091C00085FFFCCF8AE08093C4
:1094D000C60089819A81AB81BC81840D951DA61D32
:1094E000B71DB595A795979587958093B50A298956
:1094F0003A892F5F3F4F3A8B298BFD840E85EF848D
:10950000988811E001C010E05D854E853F8528896F
:10951000652F742F832F922F20E030E040EA51E432
:10952000D3D39B01AC01BD81AE81DF80C8846B2F9A
:109530007A2F8D2D9C2DA4D618166CF5EFE7FEE042
:1095400007C09091C00095FFFCCF8093C600319674
:1095500084918823B1F78091C00085FFFCCF8AE019
:109560008093C600E9960FB6F894DEBF0FBECDBF5C
:10957000CF91DF911F910F91FF90EF90DF90CF90EF
:10958000BF90AF909F908F907F906F905F904F9023
:109590003F902F9008950E94E2202B893C894D89AD
:1095A0005E89621B730B840B950B613D37E073077B
:1095B00030E0830730E0930708F440CB0E94E220BC
:1095C0006B8B7C8B8D8B9E8BE9E7FEE007C09091C7
:1095D000C00095FFFCCF8093C6003196849188230C
:1095E000B1F78091AD0A9091AE0A60E00E94A64268
:1095F000AB01BC018BE095E022E030E00E947524D5
:10960000E5E7FEE007C09091C00095FFFCCF809396
:10961000C600319684918823B1F780E090E00E94E3
:109620009A41BC018BE095E04AE050E00E949C2307
:109630008091C00085FFFCCF8AE08093C600FECAFF
:109640002F923F924F925F926F927F928F929F9252
:10965000AF92BF92CF92DF92EF92FF920F931F9340
:10966000CF93DF93C0EFDFE3C81BD90B80E090E01E
:10967000AC014F5F5F4F9A01220F331F220F331F40
:10968000F901E85BF24FA590B490CA15DB050CF028
:1096900047C0880F991F880F991FFC01E65BF24FA6
:1096A00005911491885B924FFC0185909490265B04
:1096B000324FF90165907490B801882777FD809545
:1096C000982F7DD41B012C01C819D909BE01882708
:1096D00077FD8095982F73D46B017C01601A710A15
:1096E000B301882777FD8095982F69D49B01AC0141
:1096F000C701B60197D67B018C01A818B908B5013E
:10970000882777FD8095982F5AD49B01AC01C8011A
:10971000B701BAD39B01AC01C201B101D5D217C0C8
:10972000282F2E5FCA014C33510509F0A1CF2D33EC
:1097300051F4EAE3FEE065917491882777FD809506
:10974000982F3DD404C060E070E080E090E0DF91AD
:10975000CF911F910F91FF90EF90DF90CF90BF902E
:10976000AF909F908F907F906F905F904F903F90C1
:109770002F90089580E090E0DC018093CC0A9093D4
:10978000CD0AA093CE0AB093CF0A60E070E08FE7D5
:1097900093E4209100023091010240910202509125
:1097A000030272D36093D00A7093D10A8093D20AD5
:1097B0009093D30A239A249A569A87ED80937A003D
:1097C000EEE7F0E01082808181608083808182609A
:1097D000808380818460808380818460808380E84E
:1097E00088BDEEE6F0E08081846080836AEF70E0FF
:1097F00080E090E00E94182185E090E060E00E9407
:10980000A0419093B80A8093B70A83E191E060E0A9
:109810000E94A04190930D0280930C0286E990E093
:109820000E94564290930F0280930E02089508956D
:1098300080E090E060E00E94A04180E090E0DC01E8
:109840008093B10A9093B20AA093B30AB093B40A7A
:1098500080E090E00E9456429093AC0A8093AB0A5D
:109860001092AA0A1092A90A1092B50A83E060E049
:109870000E9424221092AC0A1092AB0A1092B60AEF
:109880001092AE0A1092AD0A1092B70A1092AC0A6A
:109890001092AB0A84E060E00C942422CF93C82F8E
:1098A000E82FF0E0EE0FFF1FE158FD4F808160E0F0
:1098B0000E9424220E949520882379F5EDEAFCE09D
:1098C00007C09091C00095FFFCCF8093C6003196F1
:1098D00084918823B1F78BE095E06C2F40E050E055
:1098E0000E9466238091C00085FFFCCF8AE08093B0
:1098F000C600EBE1FDE007C09091C00095FFFCCFF2
:109900008093C600319684918823B1F78091C0007E
:1099100085FFFCCF8AE08093C600CF910895CF9356
:10992000C82FE82FF0E0EE0FFF1FE158FD4F8081B8
:1099300060E00E9424220E949520882379F5EDEAB8
:10994000FCE007C09091C00095FFFCCF8093C6005B
:10995000319684918823B1F78BE095E06C2F40E03D
:1099600050E00E9466238091C00085FFFCCF8AE012
:109970008093C600EEEEFCE007C09091C00095FF1A
:10998000FCCF8093C600319684918823B1F78091F3
:10999000C00085FFFCCF8AE08093C600CF91089578
:1099A00084E060E00E9424220E949520882309F52B
:1099B000EDEAFCE007C09091C00095FFFCCF8093DA
:1099C000C600319684918823B1F7E4EBFCE007C030
:1099D0009091C00095FFFCCF8093C6003196849192
:1099E0008823B1F78091C00085FFFCCF8AE0809387
:1099F000C60008951F920F920FB60F9211242F9355
:109A00003F934F935F936F937F938F939F93AF9306
:109A1000BF93EF93FF9380911002882331F49091CC
:109A2000B50A9093B90A91112B9A9091B90A8917A6
:109A300008F02B988F5F8F77809310028091BA0A7D
:109A4000833009F448C0843028F48130E1F082305A
:109A5000C0F50DC0853009F466C0853008F457C0E4
:109A6000863009F47CC0873009F0A6C084C010920B
:109A70007B0080E480937C0080917A0080648093F6
:109A80007A0081E01BC0209178003091790040E09D
:109A900050E08091C70A9091C80AA091C90AB0917C
:109AA000CA0A820F931FA41FB51F8093C70A909301
:109AB000C80AA093C90AB093CA0A82E08093BA0A7E
:109AC0007BC082E480937C0080917A0080648093E4
:109AD0007A0083E0F3CF209178003091790040E064
:109AE00050E08091BB0A9091BC0AA091BD0AB09150
:109AF000BE0A820F931FA41FB51F8093BB0A9093C9
:109B0000BC0AA093BD0AB093BE0A84E0D7CF1092DE
:109B10007B0081E480937C0080917A008064809354
:109B20007A0085E0CBCF209178003091790040E039
:109B300050E08091C30A9091C40AA091C50AB091E7
:109B4000C60A820F931FA41FB51F8093C30A909368
:109B5000C40AA093C50AB093C60A86E0AFCF10929C
:109B60007B0082E480937C0080917A008064809303
:109B70007A0087E0A3CF209178003091790040E00F
:109B800050E08091BF0A9091C00AA091C10AB091A3
:109B9000C20A820F931FA41FB51F8093BF0A909320
:109BA000C00AA093C10AB093C20A1092BA0A809167
:109BB000CB0A8F5F8093CB0A8091CB0A803108F467
:109BC00071C02FEF3FE38091C70A9091C80AA901A5
:109BD000481B590BCA015093AE0A4093AD0A4091FD
:109BE000BB0A5091BC0A241B350B3093B00A20935A
:109BF000AF0A21E02093B60A1092CB0A1092C70A4E
:109C00001092C80A1092C90A1092CA0A1092C30A86
:109C10001092C40A1092C50A1092C60A1092BF0A86
:109C20001092C00A1092C10A1092C20A1092BB0A86
:109C30001092BC0A1092BD0A1092BE0A20910C022A
:109C400030910D028217930744F01092AA0A1092E5
:109C5000A90A80E023DE0E945A202091AD0A3091AB
:109C6000AE0A8091B70A9091B80A8217930744F020
:109C70001092AA0A1092A90A80E051DE0E945A208E
:109C80002091AF0A3091B00A80910E0290910F029C
:109C9000281739073CF01092AC0A1092AB0A80DE0C
:109CA0000E945A20FF91EF91BF91AF919F918F91A8
:109CB0007F916F915F914F913F912F910F900FBEC8
:109CC0000F901F9018955058BB27AA270ED076C228
:109CD0003FD230F044D220F031F49F3F11F41EF413
:109CE0000FC20EF4E095E7FBDCC1E92F89D280F3C7
:109CF000BA17620773078407950718F071F49EF589
:109D0000B8C20EF4E0950B2EBA2FA02D0B01B901AD
:109D100090010C01CA01A0011124FF27591B99F0E1
:109D2000593F50F4503E68F11A16F040A22F232FED
:109D3000342F4427585FF3CF469537952795A7953D
:109D4000F0405395C9F77EF41F16BA0B620B730BE4
:109D5000840BBAF09150A1F0FF0FBB1F661F771F55
:109D6000881FC2F70EC0BA0F621F731F841F48F40A
:109D7000879577956795B795F7959E3F08F0B3CF90
:109D80009395880F08F09927EE0F9795879508957A
:109D9000DFD158F080E891E009F49EEFE0D128F09F
:109DA00040E851E059F45EEF09C0AAC162C2E92F50
:109DB000E07826D268F3092E052AC1F32617370763
:109DC0004807590738F00E2E07F8E02569F0E0251E
:109DD000E0640AC0EF6307F8009407FADB01B901F9
:109DE0009D01DC01CA01AD01EF935DD0E7D10AD03E
:109DF0005F91552331F02BED3FE049E450FD49ECF4
:109E000063CF0895DF93DD27B92FBF7740E85FE385
:109E10001616170648075B0710F4D92F96D29F93A2
:109E20008F937F936F93A9D3E0E7F0E06CD1C6D115
:109E30002F913F914F915F9101D3DD2349F09058CD
:109E4000A2EA2AED3FE049EC5FE3D0785D274DDFE1
:109E5000DF91B4C1F7D180F09F3740F491110EF437
:109E600009C260E070E080E89FE3089526F01B16C9
:109E7000611D711D811D1BC135C1EFD008F481E04A
:109E8000089575D1E395ABC10CD098C168D140F06D
:109E90005FD130F021F45F3F19F003C15111EAC1E5
:109EA0002FC1AED198F39923C9F35523B1F3951B74
:109EB000550BBB27AA2762177307840738F09F5FEB
:109EC0005F4F220F331F441FAA1FA9F333D00E2E5A
:109ED0003AF0E0E830D091505040E695001CCAF7C7
:109EE00029D0FE2F27D0660F771F881FBB1F26178C
:109EF00037074807AB07B0E809F0BB0B802DBF015F
:109F0000FF2793585F4F2AF09E3F510568F0C9C064
:109F1000B1C15F3FECF3983EDCF38695779567958A
:109F2000B795F7959F5FC9F7880F911D969587950F
:109F300097F90895E1E0660F771F881FBB1F62172E
:109F400073078407BA0720F0621B730B840BBA0BEC
:109F5000EE1F88F7E095089504D06894B1118AC186
:109F6000089556D188F09F5790F0B92F9927B7518F
:109F7000A0F0D1F0660F771F881F991F1AF0BA95CD
:109F8000C9F712C0B13081F074D1B1E0089571C148
:109F9000672F782F8827B85F39F0B93FCCF38695C3
:109FA00077956795B395D9F73EF490958095709520
:109FB00061957F4F8F4F9F4F0895E89409C097FB9D
:109FC0003EF490958095709561957F4F8F4F9F4F90
:109FD0009923A9F0F92F96E9BB279395F6958795D4
:109FE00077956795B795F111F8CFFAF4BB0F11F497
:109FF00060FF1BC06F5F7F4F8F4F9F4F16C088233E
:10A0000011F096E911C0772321F09EE8872F762F73
:10A0100005C0662371F096E8862F70E060E02AF0B4
:10A020009A95660F771F881FDAF7880F96958795A0
:10A0300097F9089507D180F09F3740F491110EF001
:10A0400019C160E070E080E89FEB089526F41B16CC
:10A05000611D711D811D2BC045C0990F0008550F52
:10A06000AA0BE0E8FEEF16161706E807F907C0F09E
:10A0700012161306E407F50798F0621B730B840BA6
:10A08000950B39F40A2661F0232B242B252B21F480
:10A0900008950A2609F4A140A6958FEF811D811D20
:10A0A000089597F99F6780E870E060E0089588233D
:10A0B00071F4772321F09850872B762F07C0662301
:10A0C00011F499270DC09051862B70E060E02AF0C2
:10A0D0009A95660F771F881FDAF7880F96958795F0
:10A0E00097F908959F3F31F0915020F48795779527
:10A0F0006795B795880F911D9695879597F908955F
:10A100009FEF80EC0895DF93CF931F930F93FF92FF
:10A11000EF92DF927B018C01689405C0DA2EEF018B
:10A120008DD1FE01E894A5912591359145915591E8
:10A13000AEF3EF01DADDFE019701A801DA9479F7B9
:10A14000DF90EF90FF900F911F91CF91DF910895D5
:10A1500000240A9416161706180609060895002406
:10A160000A9412161306140605060895C9CF50D096
:10A17000E8F3E894E0E0BB279F57F0F02AED3FE0DA
:10A1800049EC06C0EE0FBB0F661F771F881F28F033
:10A19000B23A62077307840728F0B25A620B730B56
:10A1A000840BE3959A9572F7803830F49A95BB0F3B
:10A1B000661F771F881FD2F7904896CF092E039409
:10A1C000000C11F4882352F0BB0F40F4BF2B11F4A4
:10A1D00060FF04C06F5F7F4F8F4F9F4F0895EF93D5
:10A1E000E0FF06C0A2EA2AED3FE049EC5FEB7DDD2F
:10A1F000E5DF0F90039401FC9058EDE9F0E0C7C152
:10A2000057FD9058440F551F59F05F3F71F0479527
:10A21000880F97FB991F61F09F3F79F0879508950C
:10A22000121613061406551FF2CF4695F1DF08C02B
:10A23000161617061806991FF1CF86957105610548
:10A2400008940895E5DFA0F0BEE7B91788F4BB27AE
:10A250009F3860F41616B11D672F782F8827985FF6
:10A26000F7CF869577956795B11D93959639C8F385
:10A270000895E894BB2766277727CB0197F90895BF
:10A28000ECDE08F48FEF089563DF19F068DF09F062
:10A2900037CF07CFB901CA0125CF9F775F77B0DFEE
:10A2A00098F39923B9F35523B9F3FF27951758F479
:10A2B000E52FE91BED3070F75E3B10F0F1E41CC0B8
:10A2C0009034E0F40AC0E92FE51BED3028F79E3BFF
:10A2D00010F0F1E411C0503488F4F9EA88232AF030
:10A2E0009A95660F771F881FDAF744232AF05A954C
:10A2F000220F331F441FDAF79F1B5F1BFF931F932F
:10A300000F93FF92EF9279018A01BB27AB2F9B013C
:10A31000AC0196D09701A801BF937B018C01AA27BD
:10A32000BA2FB901CA018CD0AF919701A801EF9063
:10A33000FF900F911F91D9DC41DFE1D04F9140FF99
:10A340000895552747FD509509C09B01AC0160E079
:10A3500070E080E89FE398CDA4CEC4CE59DFE8F347
:10A360009923D9F3940F511DBBF39150504094F0B1
:10A3700059F0882332F0660F771F881F91505040A4
:10A38000C1F79E3F510544F7880F911D969587951B
:10A3900097F908955F3FACF0983E9CF0BB278695F7
:10A3A00077956795B79508F4B1609395C1F7BB0FA2
:10A3B00058F711F460FFE8CF6F5F7F4F8F4F9F4FCB
:10A3C000E3CF58CF25DF58F19E5758F19851A0F0B0
:10A3D000E9F0983020F5092E9927660F771F881F1E
:10A3E000991F0A94D1F712C0062E672F782F88275D
:10A3F000985F11F4000C07C0993FB4F386957795E8
:10A4000067959395D9F7611D711D811D3EF4909557
:10A410008095709561957F4F8F4F9F4F08956894F9
:10A4200029CF27CF0BD0CACE93DE28F098DE18F0C4
:10A43000952309F036CE64CE11241CCFE1DEA0F3C3
:10A44000959FD1F3950F50E0551F629FF001729FC9
:10A45000BB27F00DB11D639FAA27F00DB11DAA1FE8
:10A46000649F6627B00DA11D661F829F2227B00D35
:10A47000A11D621F739FB00DA11D621F839FA00DC0
:10A48000611D221F749F3327A00D611D231F849F10
:10A49000600D211D822F762F6A2F11249F57504067
:10A4A0008AF0E1F088234AF0EE0FFF1FBB1F661F02
:10A4B000771F881F91505040A9F79E3F510570F0BB
:10A4C000F0CDD8CE5F3FECF3983EDCF386957795E0
:10A4D0006795B795F795E7959F5FC1F7FE2B880FB6
:10A4E000911D9695879597F908959F9340DE0F905B
:10A4F00007FCEE5F74CE11F40EF402CEF3CD88DECD
:10A50000D0F39923D9F3CEF39F57550B87FF38D05B
:10A510000024A0E640EA900180585695979528F4CB
:10A52000805C660F771F881F20F0261737074807C3
:10A5300030F4621B730B840B202931294A2BA6951A
:10A5400017940794202531254A2758F7660F771F5F
:10A55000881F20F026173707480730F4620B730B6B
:10A56000840B200D311D411DA09581F7B901842F69
:10A570009158880F9695879508959B01AC0152CF0D
:10A5800091505040660F771F881FD2F708959F9310
:10A590008F937F936F93FF93EF939B01AC0142DF07
:10A5A000EF91FF91B0DD2F913F914F915F913ACFA5
:10A5B000629FD001739FF001829FE00DF11D649FA7
:10A5C000E00DF11D929FF00D839FF00D749FF00D33
:10A5D000659FF00D9927729FB00DE11DF91F639FD4
:10A5E000B00DE11DF91FBD01CF011124089597FBA6
:10A5F000092E07260AD077FD04D049D006D00020C6
:10A600001AF4709561957F4F0895F6F790958195AE
:10A610009F4F0895A1E21A2EAA1BBB1BFD010DC07E
:10A62000AA1FBB1FEE1FFF1FA217B307E407F50702
:10A6300020F0A21BB30BE40BF50B661F771F881FDE
:10A64000991F1A9469F760957095809590959B0174
:10A65000AC01BD01CF01089597FB092E05260ED050
:10A6600057FD04D0D7DF0AD0001C38F45095409530
:10A67000309521953F4F4F4F5F4F0895F6F79095D6
:10A680008095709561957F4F8F4F9F4F0895AA1BBE
:10A69000BB1B51E107C0AA1FBB1FA617B70710F0CD
:10A6A000A61BB70B881F991F5A95A9F780959095FF
:10A6B000BC01CD010895EE0FFF1F0590F491E02D30
:10A6C0000994A1E0B0E0E6E6F3E576C55B0161152B
:10A6D000710521F0DB018C9311969C93482F592F23
:10A6E0006A01F601E1906F018F018E2D90E080D21A
:10A6F0000097B9F7FE2DFD3229F4D601ED908D01BA
:10A7000021E007C0BE2DBB3219F4F601E1908F01A4
:10A7100020E068010894C108D108C60163EA7FE01F
:10A7200043E050E029836CD22981009709F572E05B
:10A73000E72EF12CE00EF11EC70166EA7FE045E04E
:10A7400050E05ED22981009729F467E0E62EF12CD3
:10A75000E00EF11EA114B10421F0D5011196FC9276
:10A76000EE9220FF0AC130E020E090E88FEF0DC1AB
:10A77000C6016BEA7FE043E050E0298341D22981A2
:10A78000009731F060E070E0CB01662477240AC0C6
:10A79000A114B10409F4F5C00E5F1F4FF501118338
:10A7A0000083EFC03E2D30533A30A0F52260E22FF7
:10A7B000F0E0AF014870507022FF07C0411551050D
:10A7C00071F50894611C711C2AC04115510519F0DE
:10A7D0000894610871086B017C0152E0CC0CDD1C0F
:10A7E000EE1CFF1C5A95D1F76C0D7D1D8E1D9F1D13
:10A7F000660F771F881F991F630F711D811D911DA3
:10A800006839F9E97F07F9E98F07F9E19F0738F01F
:10A81000246005C03E3F39F423FD3FC02860D801C5
:10A82000ED908D01BFCF353311F03531B1F5F80121
:10A8300031913D3211F4206102C03B3241F4D80124
:10A8400011963C911197319642E050E002C041E0F0
:10A8500050E030533A3020F08F01041B150B1DC01F
:10A8600040E050E0BCE040385B075CF4DA01AA0F3E
:10A87000BB1FAA0FBB1F4A0F5B1F440F551F430F7F
:10A88000511D319130538F013A3060F324FF03C0E2
:10A89000509541955F4F640E751EC22EDD2421FF39
:10A8A00008C0A114B10429F001501040F501118332
:10A8B000008383DB7B018C01F3E0CF22DD2433E0D6
:10A8C000C316D10421F417FB109517F91095C80190
:10A8D000B70120E030E0A901D0DA882309F448C0AC
:10A8E00077FE09C042ECC42E4FE0D42E70946194E0
:10A8F0007108739404C03AEDC32E3FE0D32E26E0D6
:10A90000822E912C90E2A92EB12C0EC0F601259139
:10A91000359145915491C801B70184DDE62EF72E9B
:10A92000082F192F6A187B086A147B047CF7B594EA
:10A93000A7940894810891088114910429F08CEF60
:10A940009FEFC80ED91EF0CFB701C801282F220FE4
:10A95000292F221F2F3F31F020E030E0A9018DDAAE
:10A96000882331F482E290E09093F60A8093F50A0E
:10A970003E2D2F2D902F812F08C030E020E090E851
:10A9800003C030E020E090EC8FE7F901AC016F2FBD
:10A99000722F852F942F2196EEE02AC42F923F929A
:10A9A0004F925F927F928F929F92AF92BF92CF927F
:10A9B000DF92EF92FF920F931F93CF93DF934B01A0
:10A9C000EA016115710519F0FB01808391832097DD
:10A9D00039F09E01225030402332310508F0F1C099
:10A9E000A82EB92EF50111915F017F01812F90E012
:10A9F000FFD00097B9F71D3229F4F50111917F01BD
:10AA000001E006C01B3219F4F50111917F0100E04D
:10AA1000209719F0C031D105B9F4103381F4F70152
:10AA20008081883711F0883551F4F701118182E077
:10AA300090E0E80EF91E0260C0E1D0E005C020976A
:10AA400019F41033C1F422C0C830D105F9F0C9306F
:10AA5000D10524F4C230D10509F507C0CA30D105AB
:10AA600051F0C031D105D1F426C0A12CB12CC12C9C
:10AA7000F0E4DF2E25C0CAE0D0E0ECECAE2EECEC2A
:10AA8000BE2EECECCE2EECE0DE2E1AC0C8E0D0E0FC
:10AA9000A12CB12CC12C70E1D72E12C09E014427ED
:10AAA00037FD4095542F60E070E080E090E8B2DD23
:10AAB00059016A0105C0A12CB12CC12C68E0D62E29
:10AAC00040E060E070E0CB011E01442437FC40947C
:10AAD000542C50ED752E710EE72DEA3070F0212FB9
:10AAE00021542A3118F439EC732E06C0212F215637
:10AAF0002A3128F529EA722E710E272D30E02C1705
:10AB00003D07ECF447FD17C0A616B706C806D906E0
:10AB100078F0A20191014CDD670D711D811D911D21
:10AB20006130F0E07F07F0E08F07F0E89F0710F05A
:10AB30004FEF01C041E0F70111917F01CACF8114AD
:10AB4000910491F0442339F00894E108F108F401EC
:10AB5000F182E08209C001FF1BC097012250304002
:10AB6000F4013183208314C047FF12C000FF05C0E9
:10AB700060E070E080E090E804C06FEF7FEF8FEF5F
:10AB80009FE722E230E03093F60A2093F50A16C0E0
:10AB900000FF08C090958095709561957F4F8F4F0D
:10ABA0009F4F0CC097FF0AC082E290E09093F60A94
:10ABB0008093F50A6FEF7FEF8FEF9FE79B01AC016A
:10ABC00003C020E030E0A901B901CA01DF91CF91B3
:10ABD0001F910F91FF90EF90DF90CF90BF90AF90BB
:10ABE0009F908F907F905F904F903F902F9008950F
:10ABF00091113BC2803219F089508550D0F70895E9
:10AC0000FB01DC014150504088F08D9181341CF0F3
:10AC10008B350CF4805E659161341CF06B350CF45F
:10AC2000605E861B611171F3990B0895881BFCCF40
:10AC3000FC018191861721F08823D9F7992708957F
:10AC40003197CF010895FB0151915523A9F0BF0120
:10AC5000DC014D9145174111E1F759F4CD01019007
:10AC6000002049F04D9140154111C9F3FB014111FC
:10AC7000EFCF81E090E001970895AEE0B0E0E2E42C
:10AC8000F6E5A4C20D891E8986E08C831A830983A8
:10AC90008FEF9FE79E838D839E01275E3F4FCE01FE
:10ACA00001966F89788DA90108D0EF81F885E00FB2
:10ACB000F11F10822E96E4E0A5C2ACE0B0E0E2E61F
:10ACC000F6E576C26C011B018A01FC01178216822F
:10ACD000838181FFC4C12E010894411C511CF601DF
:10ACE0009381F10193FD859193FF81911F01882349
:10ACF00009F4B1C1853239F493FD859193FF8191B7
:10AD00001F01853221F490E0B601C8D1E8CFEE24CE
:10AD1000FF2420E02032B0F48B3269F08C3228F42A
:10AD2000803251F0833271F40BC08D3239F08033B0
:10AD300049F421602CC02260246029C0286027C00B
:10AD4000206125C027FD2CC0382F30533A3098F4AD
:10AD500026FF08C08E2D880FE82EEE0CEE0CE80EB4
:10AD6000E30E15C08F2D880FF82EFF0CFF0CF80E88
:10AD7000F30E20620CC08E3221F426FD6CC12064DB
:10AD800006C08C3611F4206802C0883649F4F101FF
:10AD900093FD859193FF81911F01882309F0BACF1C
:10ADA000982F9554933018F09052933028F40C5FFC
:10ADB0001F4FFFE3F9830DC0833631F0833771F005
:10ADC000833509F05CC021C0F801808189830E5F62
:10ADD0001F4F420171E0A72EB12C15C062E0662E14
:10ADE000712C600E711EF8018080918026FF03C0D7
:10ADF0006E2D70E002C06FEF7FEFC4012C8743D14E
:10AE00005C0183012C852F7716C052E0652E712CD2
:10AE1000600E711EF8018080918026FF03C06E2DA8
:10AE200070E002C06FEF7FEFC4012C8721D15C017D
:10AE30002C852068830123FD1EC007C080E290E0BE
:10AE4000B6012C872BD1FA942C858F2D90E0A81673
:10AE5000B906A0F310C0F40127FD859127FF819169
:10AE60004F0190E0B6012C8719D12C85F110FA948E
:10AE70000894A108B108A114B10469F7E9C08436A7
:10AE800011F0893641F527FF08C0F8016081718112
:10AE9000828193810C5F1F4F09C0F801608171812D
:10AEA000882777FD8095982F0E5F1F4F4FE6B42EB1
:10AEB000B22297FF09C090958095709561957F4F5C
:10AEC0008F4F9F4FF0E8BF2AA2012AE030E012D155
:10AED000782E741844C0853731F43FEEB32EB22279
:10AEE0002AE030E025C099EFB92EB2228F36C1F0AA
:10AEF000803720F4883509F0AEC00DC0803721F0CE
:10AF0000883709F0A8C002C020E1B22AB4FE0BC005
:10AF100084E0B82A08C0B4FE09C0E6E0BE2A06C034
:10AF200028E030E005C020E130E002C020E132E05E
:10AF3000B7FE08C0F80160817181828193810C5F46
:10AF40001F4F07C0F8016081718180E090E00E5FC3
:10AF50001F4FA201CFD0782E7418FFE7BF22B6FE94
:10AF60000BC02EEFB2227E1438F4B4FE07C0B2FC40
:10AF700005C08FEEB82202C0A72C01C0AE2C8B2DCD
:10AF800090E0B4FE0DC0FE01E70DF11D20812033DD
:10AF900019F4E9EEBE2209C0A394B2FE06C004C0B3
:10AFA00086789070009709F0A3948B2C9924B3FCB9
:10AFB00013C0B0FE0EC0AF1428F4E72CEF0CEA1853
:10AFC000AF2C07C0E72C05C080E290E0B60166D048
:10AFD000A394AF14C8F304C0AF1410F4FA1801C05E
:10AFE000FF2484FE0EC080E390E0B60157D082FEBD
:10AFF0001DC081FE03C088E590E010C088E790E0A6
:10B000000DC0C40186789070009781F081FC02C069
:10B0100080E201C08BE2B7FC8DE290E0B6013ED049
:10B0200005C080E390E0B60139D0EA947E14C8F3FD
:10B030007A94F201E70DF11D808190E0B6012ED0E7
:10B040007720B1F705C080E290E0B60127D0FA94EE
:10B05000FF20C9F744CEF6012681378102C02FEFC9
:10B060003FEFC9012C96E2E1BFC0992788270895D8
:10B07000FC010590615070400110D8F780959095C3
:10B080008E0F9F1F0895FC016150704001900110C8
:10B09000D8F7809590958E0F9F1F08950F931F935B
:10B0A000CF93DF938C01EB018B8181FF1BC082FF6B
:10B0B0000DC02E813F818C819D812817390764F452
:10B0C000E881F9810193F983E88306C0E885F98571
:10B0D000802F0995009731F48E819F8101969F837F
:10B0E0008E8302C00FEF1FEFC801DF91CF911F9138
:10B0F0000F910895FA01AA27283051F1203181F1EA
:10B10000E8946F936E7F6E5F7F4F8F4F9F4FAF4F6F
:10B11000B1E03ED0B4E03CD0670F781F891F9A1F82
:10B12000A11D680F791F8A1F911DA11D6A0F711D36
:10B13000811D911DA11D20D009F468943F912AE042
:10B14000269F11243019305D3193DEF6CF0108952A
:10B15000462F4770405D4193B3E00FD0C9F7F6CF5B
:10B16000462F4F70405D4A3318F0495D31FD405223
:10B17000419302D0A9F7EACFB4E0A69597958795B9
:10B1800077956795BA95C9F7009761057105089598
:10B190009B01AC010A2E0694579547953795279544
:10B1A000BA95C9F7620F731F841F951FA01D0895DC
:10B1B0002F923F924F925F926F927F928F929F92C7
:10B1C000AF92BF92CF92DF92EF92FF920F931F93B5
:10B1D000CF93DF93CDB7DEB7CA1BDB0B0FB6F89466
:10B1E000DEBF0FBECDBF09942A88398848885F84A6
:10B1F0006E847D848C849B84AA84B984C884DF8017
:10B20000EE80FD800C811B81AA81B981CE0FD11DFA
:10B210000FB6F894DEBF0FBECDBFED010895F894D0
:02B22000FFCF5E
:10B222005573696E672044656661756C7420736539
:10B232007474696E67733A004D31313000482000F2
:10B242004C20002569206D696E2C202569207365CC
:10B2520063004D31303420496E76616C696420653B
:10B262007874727564657220004D31303520496EF4
:10B2720076616C6964206578747275646572200009
:10B282004D31303920496E76616C6964206578747D
:10B29200727564657220003F006F6B0020703A0087
:10B2A20020693A0020643A0020633A005400496E53
:10B2B20076616C69642065787472756465720041A8
:10B2C20063746976652045787472756465723A2094
:10B2D200002E00537465707261746520746F20686B
:10B2E200696768203A2000504944204175746F74A0
:10B2F200756E652073746172740000803B45008036
:10B302003B4500007043000000006400640060EAF6
:10B3120000000080BB44010101010101713DE841CF
:10B32200A97E443E756089440000803FFF3FFF3F95
:10B332000158595A45000001001A0019000A00007C
:10B3420000FFFF1C001B000A000100FFFF17001690
:10B35200000A000200FFFFFFFFFFFF04000E0018BB
:10B362000015000A0003000000010002000200288C
:10B3720023000028230000640000001027000000C2
:10B3820000FA430000FA430000A0400000344200EB
:10B3920000A04214AE9F4200002045F6C8154403A7
:06B3A20000480D3D000013
:00000001FF
